:10000000020061C0E0C083C082907004E002460933
:100010000000000239D000004003901218544F59DC
:100020004548410000023BC15558310000023C0ADE
:10003000436F7079726967687420284329203139C9
:100040003930204F4B4920456C65637472696320D9
:10005000496E64757374727920436F2E2C4C7464EE
:100060002EC2AF75B0FF7590D775C0007807D8FE67
:10007000C2B590700474EFF0907001E4F075EE0476
:100080007581CF740D90D000F090D0037407F0000C
:10009000740090D001F0741A90D004F0744090D0A5
:1000A00005F074CD90D000F012049E90FF00E4F8AB
:1000B000FFEF9328F8DFFAD583F7EF9328F8DFFAFC
:1000C000E860057B010203C578FFE4F6D8FD90C027
:1000D00000780112079960057B020203C512073DF3
:1000E00060057B040203C590BEBEE0B44114A3E0EA
:1000F000B4450FA3E0B4490AA3E0B44F05D20A0205
:10010000012E90BEBE7441122F82A37445122F821D
:10011000A37449122F82A3744F122F8212057312F7
:10012000054212057A1205C412072D124E3A90BFED
:100130002CE07002740190C0FFF01207D560057BBF
:10014000030203C590BF2CE0F91231EC1204C290F7
:10015000C0FAE0A2E4923D7526EF757D3E7554002D
:10016000755277123322D21D740BF556F55590BF98
:10017000337F04E054384FF557F454384446F5259E
:10018000752401755300E52512330575C80075CA3D
:100190007075CBFE758805758AC0758CB4758BB388
:1001A000758DFF75894075F84075B801907000F045
:1001B00075A8B575C80475985075D90490D002E03B
:1001C00054807003437A8090C060E5EDA2E7E4506C
:1001D00001F4F0927B90D003C2AFE04410F0D2AFB4
:1001E000C2DAC2DBD2D8E5D830E1FBE5DC90C096BC
:1001F000F090D003C2AFE054EFF0D2AFD217D2707C
:1002000074031204D0D27375710578C476157570B5
:10021000FF7F017490122F6878C4E6602A122E0ABC
:1002200050F6F5727F0F7490122F68E572B4500388
:10023000020236B4510990BF71122F820202547526
:1002400070FFD571CC800274FF90BF71122F827B3A
:10025000070203FFC2687402122F5912044075543A
:100260004443551075570012324D122E0A78D2E6CB
:10027000086670F3741E78C3F674031204D0C27358
:1002800074051204D0D27D7571021233B97F0174E6
:1002900090122F6878C4760B78EF7600757200D2D2
:1002A00069122E0A78EFE6700F78C4E670F3E572F3
:1002B000703AD571D50202CC78EF7600F572FF1254
:1002C000080D60DDEF64F1700302037890BF727473
:1002D000FF122F82C269C27DC22EC268C27478DB4F
:1002E00076007F0F7490122F68020322C269E572B4
:1002F00090BF72122F827F0F7490122F68122E0AF5
:1003000012324D78C3E670F5D22ED2687402122FE5
:1003100059120440755444435510755700741478AD
:10032000C3F6122E0A12324D78C3E670F5D27375F9
:10033000550075540075570012045290BF72E0B416
:100340004008E57A30E7030203C078CA760778CE22
:100350007615785E7F1C12301B12497312071C90B1
:10036000BF34E4122F8290BEB9E4122F8290BEBA3D
:100370007402122F82021A63D273C27D90BF72EF91
:10038000122F82755500755400755700C26AD24706
:1003900074907F00122F687400122F5974407F00F0
:1003A000122F6874A07F00122F68740A1204DA906A
:1003B000BEBBE4122F82E57390BEBD122F82C273C2
:1003C000D27D0209B11204C2740BF556F55575C8F9
:1003D0000075CA7075CBFE758805758AC0758CB4BA
:1003E000758BB3758DFF75894075F84075B80190B0
:1003F0007000F075A8B575C80475985075D9048B50
:100400007374151204D0D273D27D742F122F59E554
:1004100073122EA5C26AC26DD2477F007490122F4C
:100420006875240175530075257E12049E1233B938
:10043000122E0A50F8B434F5E573B403F002010249
:10044000D26AD2477F0574A0122F687FFF744002E2
:100450002F687F0074A0122F687F027440122F68EB
:1004600074227F08122F6890BF5FE0601B90BF5E10
:10047000E0A2E472E092E0122F8230E00B755D188A
:10048000743F122F5902048B1249A4D211C2107565
:1004900058027F007490122F68D26AD247227401EA
:1004A0001232DD74001232F3747E023305752401BA
:1004B000755300752546E557F454384525F5250252
:1004C0003305747878D0F608F674A008F608F6229A
:1004D000122E0A78C4F6B600FD2278C4F6122E0A4F
:1004E00012324D78C4E670F52278767F0412301B04
:1004F00090BEC3E0600B7B007C067D557E36120506
:100500005AA3E0600B7B007C007D027E5612055AE8
:10051000A3E0122FC97B007C00FEADF07401120530
:100520005A787690AF2B7A04E6540F7003740AD68B
:10053000E6B41000500244A0122F8212309708DA5D
:10054000E72290BEBBE4122F821207E690BF2CE098
:10055000F91231EC1204E9020802FF7879E62ED490
:10056000F618E63DD4F618E63CD4F618E63BD4F689
:10057000DFE9229070057401F0229070057400F09C
:100580002200000000000000014E000F00000000EB
:10059000000000014E000F00000000000000014EAE
:1005A000000F00000000000000014E000F000000DE
:1005B00000000000014E000F0A12340E00123456E3
:1005C0007800005590BF1E7A0512072390A06BE0BB
:1005D00013B3E492E090BF2D122F8290BF2CE4124F
:1005E0002F8290BF2E7A0212072390BF3074181208
:1005F0002F8290BF317418122F8290BF327418125C
:100600002F8290BF337418122F8290BF6C7A05121C
:10061000072390BF36E0E4122F8290BF37E4122FF9
:100620008290BF73E4122F8290BF38E4122F829021
:10063000BF34E0E4122F8290BF39740A5403122FA2
:100640008290BF5EE4122F8290BF5F7404122F82EB
:10065000125A4F7412122F82125A4F7434122F8270
:10066000125A4FE4122F82125A4FE4122F82125A5A
:100670004FE4122F82125A4F74B6122F8290BF3A53
:100680007A0312072390BF3D7A0F12072390BF4CC5
:100690007A0F12072390BF247A0312072390BF27F3
:1006A000E4122F8290BF5BE4122F8290BF5C741320
:1006B000122F8290BF5DE4122F82757EC8125A5E9F
:1006C000757EC9125A5E757ECA125A5E757ECB124D
:1006D0005A5E757ECC125A5E757ECD125A5E90BE01
:1006E000B8E4122F8212587C90BEB9E4122F829087
:1006F000BEBA7402122F8290BEB7E4122F8290BF4E
:1007000023E4122F8290BEC77A0A12072390BED22A
:100710007A0812072390BF74E4122F8290BEC6E4B9
:10072000022F82E4122F82125A4FDAF72290BEAFC4
:100730007A087420122F82125A4FDAF622786490C7
:10074000A2AAE0F60890A72AE0F60890A3EAE0F64D
:100750000890A16AE0F60890A6AAE0F60890A22AFE
:10076000E054F0F67A2078697F017D0A12300AE5BC
:100770006330E006636453636590DAEAE5644565D7
:100780007016E5606481701090BEC278607904E6EE
:10079000122F82A308D9F8E422122DFCE8FFE4F01E
:1007A000A3B582FADFF8122E01E8FFE0F4F0A3E42B
:1007B000B582F8DFF6122E01E8FFE064FF7015F055
:1007C000A3B582F6DFF4122E01E8FFE07006A3B5B0
:1007D00082F9DFF72290A02B78007F43E028F812FF
:1007E0003097DFF8E82290A02B7A417800122DFC98
:1007F000900581E893122E01122F8212309708DAA9
:10080000EC22125C7590B0AB7455022F82FF64022B
:100810006017EF64406012EF6450600DEF64516048
:1008200008EF64536003EF64D02278EEB60002C391
:1008300022E6B40800400302098914900841020B23
:100840006C02085602086702088B0208B5020923E9
:1008500002093402099478D2E60866700778C476F3
:100860000378EE0602099278C4E6601CC27378EF42
:100870007600D27D7F017490122F6878C4760B7851
:10088000DB7600D26978EE0602099278C4E6600D44
:1008900078EFE6601D12080D60180208CC78EFE6CC
:1008A000703C7F017490122F6878C4760BD26978FF
:1008B000EE0602099278C4E6600D78EFE6606112F8
:1008C000080D605C0208CC78EFE6701290BF72747D
:1008D000FF122F827F0F7490122F6802091A78EF8F
:1008E000E690BF72122F827F0F7490122F68E55826
:1008F0006006FF7440122F68E5596006FF745012BD
:100900002F6830740A7F0C301C027F0B122F3AE5DF
:100910007F541060057F07122F3AC26978EE760582
:1009200002099278D2E60866700778C4760378EEFA
:100930000602099278C4E6705990BF72E0B4FF0FC6
:10094000C27DC22EC268C27478DB7600020989D2E9
:100950007DD268D243D26AD247307406301C03433A
:100960007F20D2737F007490122F6890BF72E06472
:10097000026016124969124C17125CB86008743F85
:10098000122F5902098912511AD2735355EF78EE7A
:100990007600D32290BF74E0B40104C26AD24790BB
:1009A000BF7274FF122F8278DB760078EE7600D368
:1009B000221233997F007490122F68537A8090BF6F
:1009C00072E064F16028437A40122E9EE4122F599F
:1009D0007FFF8F587440122F687F0074508F591218
:1009E0002F687F0590C0F3EFF074A0122F68433991
:1009F000F012333079B97707B700FD123347533F10
:100A00000F1234DB123232E4F55212343D12347DCF
:100A100075550DD268D22E1234A11232C1785C7F86
:100A20001E12301B537AF71233B91232891214EFA7
:100A30005000122E0A50F0FF1214EF4031EFF55C17
:100A4000C41215AEE55C1215AE785EE6640260086D
:100A5000E6186670D2020B51E55F24A640BFE55F41
:100A60009016219360EFF460B4F4F55D80B9CF5433
:100A70003FCFBF170050B030E10B20E3088F5C90F0
:100A80000A88EF2F73020B2180E2802A804F805367
:100A90008057805B8060806280648066806880CCE4
:100AA000806880C8807280C480C2806F80BE80BC35
:100AB00080BA80B880B6A21F74073400F55C122E8D
:100AC0009E740C122EA5E55C122FC9122EB97F2D33
:100AD0007418122F68437A08E55C020A40A22A744F
:100AE0000B80D7A229740D80D1A21E741080CBA2D6
:100AF00028B3744180C4742080C2740A80BE742AF2
:100B000080BA744980B6740980B2122E9E740C1299
:100B10002EA5437A08020A27020A27122E9E0214E3
:100B20008912152EB405005025FF900B30020A8261
:100B30008008801D80E280E38014E55E6402700E10
:100B4000E55F122FD8F55F7F2D7418122F68020A07
:100B500027E55F24A64012E55F90167B25E0FF9312
:100B6000CF04938F83F582E473021489FF2F2F73D0
:100B70001214EF40097970A7607E010214C70214B5
:100B80008912333079B97707B700FD123347123332
:100B900022537ADF020A04854070853F7153710742
:100BA000E55154030303A21E92E3A21F92E4427193
:100BB000123138E55233C4A23E92E3A23F92E2A240
:100BC0002A92E1A22992E0F57279707E030214C79D
:100BD000C2AF1233BCD2AF021489D27E0214891282
:100BE000333079B97707B700FD123347533F0F12FF
:100BF00034DB1234000214891234050214891214F1
:100C0000EF502985603F856140C37405955E400DB6
:100C10000475F004A4FF783F7D02122FF97840128A
:100C20002FE5F53F8E401234DB0214898560408544
:100C3000613F80F21214EFE5605001C47852D6E6AD
:100C400012343D0214891234850214891234890247
:100C5000148912348D0214891234910214891236C7
:100C600080021489C222E5241232DDC21E75302AA8
:100C70000214891214EFE5605001C4540FB403004C
:100C8000501B2323907004C2AF5326F34226E5265F
:100C9000F0D223D2AFE5241232DD021489C223E55B
:100CA000241232DD0214891214EFE560500F602423
:100CB000B420004008540F1230310214891230372A
:100CC000F5531232F3432430E5241232DD740DF56E
:100CD000550214891234A15324CF80EC748080E033
:100CE000744480DC12370E021489123715021489FD
:100CF00012333079B97707B700FD123347021489F0
:100D000012336902148912336912337F1233B91214
:100D100015F5600A20AAF53039F2C23980EE123397
:100D20009912333079B97707B700FD123347020AB9
:100D3000041214EFE5605001C4C40354385325C7AE
:100D40004225E525123305021489856024E5241225
:100D500032DD021489E560B49004E5908013B4B0EC
:100D600004E5B0800CB4C004E5C08005B4ED0AE52C
:100D7000ED7970F77E010214C7021489AF60E56156
:100D8000BF900EA2E59295A2E49294A2E392938082
:100D90000EBFB006A2E492B48005BFC002F5C00247
:100DA00014891236447970F77E010214C785608376
:100DB0008561821214EF4012E5837005A982E780F5
:100DC00001E07970F77E010214C785837085827116
:100DD000122E9EE570122ED5E571122ED5E570B457
:100DE0000006E571F9E78007857083857182E0125E
:100DF0002EB91233B9122E0A50F8543FB40B09859C
:100E00007083857182A380C2B40C111571E571B431
:100E1000FF02157085708385718280AEB411D30294
:100E2000148990BEBB809AA860A961E562B80003EE
:100E3000F7800788838982122F820214891214EFA7
:100E400040277A1F90A02B858370858271E0FF7404
:100E500014122F68857083857182123097DAE8E06A
:100E6000FF741C122F68020A1D90A02B85837085C9
:100E70008271122E9EE570122ED5E571122ED58547
:100E80007083857182E0122EB91233B9122E0A5086
:100E9000F8543FB40B0B85708385718212309780B4
:100EA000CBB40C0280C3B411E00214891214EF40D9
:100EB000299070057401F090A02B757243858370A2
:100EC0008582711214F4857083857182122F8212CB
:100ED0003097D572E8907005E4F002148990BEC294
:100EE00079707F04E0F7A309DFFA79707E040214B9
:100EF000C71233E60214891233EF0214891233F554
:100F000002148979769000177805E893F719D8FAD2
:100F100090BF71E0F719A3E0F71214EF4007797260
:100F20007E020214C779707E070214C7E4F570F5DB
:100F300071F5721236C612372E1233B9103C0C12EC
:100F400015F570F579707E020214C7123801700F22
:100F5000787204B6000206041826F618E436F68005
:100F6000D8E4F570F571F5721236D612372E1233B9
:100F7000B91237C614600F1460071215F570EF80B0
:100F8000C312387580E878710426F618E436F680C6
:100F9000DD788A7F1F12301B75708A755D1F1214F1
:100FA000F44012A9700570F7D55DF31214EF5015D7
:100FB0001214F450FB122E9E020FC5798A777C0919
:100FC0007E0512160C75330512368D123289301BD0
:100FD000FA123405C21B1232890214897860798BA7
:100FE0007F0C123023020FEF798B7E0212160C75E4
:100FF00033021236B278301233B9123289B62AF778
:101000001232891232320214891236C612372E7504
:1010100070001233B91237736050123825123741FD
:10102000605D7970B7000CB44040070978831230D6
:101030002180DFB480341214EF400E79717E0512E6
:1010400014D279837E050214CC122E9E79717E050E
:10105000E7122ED509DEF9E4122F591233B9121511
:10106000DE70F879837E050214DE1215DE70A37936
:1010700070E777427E01600477437E060214C779E9
:10108000837E050214C71236D612372E1233B912D8
:1010900015DE600B1237C6B402F212387880E079A0
:1010A0007077427E010214C7798A7763097E0578DA
:1010B00060123021DEF975330512368D437A200235
:1010C0000A1D8560708561718562721214EF500C83
:1010D00078707903E6122FD8F608D9F87819E572F6
:1010E0007002887212333079B97707B700FD123376
:1010F0004785727478C47664857073123400123335
:10110000B9122E0A5011FF1214EF743D5006CF543D
:101110003FCF74116F601B78C4E670E27664D574BB
:10112000DD857274D573D7301FCE85717312340587
:1011300080CC123405021489FF00AA55CC33816992
:10114000AF1278707F0812301B798B7F0A901138AC
:10115000E493F709A3DFF912333079B97707B700C1
:10116000FD123347D222C223E5241232DD123400AD
:10117000537ADF437A1075305A1236C612372E1260
:1011800033B9123289103C081215F570F20211E7DA
:1011900090C000E534B40A00500375820A7F0B79D1
:1011A000A3E0F7A309DFFAE5356008FF78AD7D0B12
:1011B00012300A788B79A37E0A7A00E6677F0833BB
:1011C00050010ADFFA0809DEF27972EA1211F479A5
:1011D0007574011211F4E7640070A409E7640470E7
:1011E0009E09E764E27098537AEF12323279707E8A
:1011F000060214C727F719E437F719E437F72278FE
:1012000061122FE5F570EEF5717863122FE5F57236
:10121000EEF573E5647002740CF57478C476158588
:10122000703F8571407576001234DB122E9E122EAF
:10123000DF8574751233B9122E0A4026E57670F4F4
:1012400078C4E670EF7615D575EAC3E5409573E589
:101250003F957250CA74012540F540E4353FF53F93
:1012600080C6F81214EF74065010C8543FC8740BAF
:101270006860AC740C68600874116870B7021489F7
:1012800074FF627680AE7861122FE5F5708E71780A
:1012900063122FE5F5728E73E5647002740AF574BB
:1012A00075770078C4760485703F85714075760047
:1012B0001234DB122E9E122EDF8574751233B91292
:1012C0002E0A401DE57670F478C4E670EF7604D5FA
:1012D00075EA6377FFE57760CE85723F857340805E
:1012E000CCF81214EF74065010C8543FC8740B6841
:1012F00060B5740C68600874116870C00214897459
:10130000FF627680B71214EF4007C273C2AC0213BB
:101310001874B07F01122F6874FFF572F56DF56EC9
:10132000755E201233B930980AC298E5997973F73F
:101330001213C5122E0A50EBFF1214EF401AE57279
:1013400060077572008F6D80DAEF556D64FF605B2A
:101350007572FF8F6E021374CF543FCFEFB4170036
:1013600050C19013AE9320E7BA20E63F20E5051266
:1013700015AE80AFE56DF59979B97708B700FDE551
:101380006EF59979B97708B700FD1214EF509412F1
:101390002E9EE56D122ED5E56E122ED57E07742D8C
:1013A000122EDCDEF9122F58021323021489800159
:1013B0000203040506070809000A0B20400E800CF2
:1013C0000E0D80800F1214EF400A7973E7FF74143A
:1013D000122F6822122E9E7973E7122ED5747CB7D5
:1013E0003F027480B71F005004E72727277E04FAC6
:1013F0009013FF93122EDC0AEADEF4122F58224ECD
:101400004F4F502031202020322020203320202018
:101410003420202035202020362020203720202076
:10142000382020203920202030202041535452538E
:1014300048525053454E4420454E44204C4F43485B
:101440004F524E20434C52205354522052434C444E
:101450004F574E2055502046554E43204F4E482062
:101460004F46485F5F5F5F202020202020202041E2
:101470004C50485352434820202020202020204E0A
:101480004E4C54437A020214891214EF5003121482
:1014900094020A1D122E9EA21F1214C1A22A121417
:1014A000C1A2291214C1A21E1214C1A228B312147F
:1014B000C1E551122EC3E5525407122EC3122EDF7E
:1014C00022E43400022EC31214EF40121214D2028E
:1014D0000A1D75F014E7FF122F6A09DEF822122E9A
:1014E0009EE7122ED509DEF9E4122F59020A1DE5F6
:1014F0007AA2E622537AF31233B9122E0A50F8FF79
:101500001214EFEF501D543FFF12152560051470A3
:10151000E6D3227408627A557A70DCE55EC3132440
:101520005EF8E6C322EFB41200506502153EEFB438
:101530001200505CB40C005005E57A30E352EF9095
:101540001545020A8280498020801E801C801A80F6
:10155000188016802480228020802E8030803D805C
:10156000328033802B80298030E55EC394024009AD
:10157000E57A30E204EF2409FFEFF55C122EA5E5D1
:101580005C1215AE537AFBE4227F0080EC637A0490
:10159000740422740122740222740322E57A20E387
:1015A0000B122E9E740C122EA5437A0880E2785EF0
:1015B000B62000500AF5F0795FE61215CC062278C5
:1015C0006E7F10C4D6C4C618DFFA80F2C31392D55A
:1015D00029F9E5F0540F20D503C4F722D722122EA3
:1015E0000AF87401500E1214EF74385006C8543FB4
:1015F000C874116822122E0AF87401500E1214EFEA
:10160000741F5006C8543FC8741168227F06901694
:101610001BE493F709A3DFF9DEF222FF00AA55CC01
:1016200033FF00000000040000000604000000007A
:101630000000000000000000000006FFFF0000FFA7
:10164000FF04000E00000000FFFFFF04000C00007C
:101650000000FFFF06040008FF00FFFFFF06000078
:101660001A0000000404FFFFFF000C04000000FF4C
:101670000000040A040408FFFFFFFF14890B810027
:10168000000B970BD00B700B810BDF0BF80BFE0CD4
:10169000340C460C4C0C520C580BDA0C5E0C640FDC
:1016A000BB0FE8100910860E3D0F030EDD0DAD14C3
:1016B0008914890F2C0F61148914890C730C9D10E7
:1016C000A80CDC0CD40CE00CD41489148914890CFB
:1016D000A70CD412860CF00D000D060EAC14891464
:1016E000890D7C0D550DA20E2714890E2214891424
:1016F00089148910C214890F910FDC10090CE40CB5
:10170000EA0D310D4A148914891489114211FF130D
:10171000050EF10EF70EFD1489148319E819081946
:101720006E17D2172F18A41489148914891489E507
:101730006054C0600302148985607090D001E05449
:10174000C04402121900440812190074804570FA4E
:101750001218EE54F71219007571007572007F109F
:1017600090D002E0A2E5E57233F572E57133F571D0
:1017700090D001E0121901DFE74404F054FDF05469
:10178000FBF04404F04402F01214EF400779717E3C
:10179000020214C7122E9EE570122ED5E571122E8C
:1017A000D5E572122EB91233B9122E0A50F8543FF1
:1017B000B40B05E570048006B40C0AE57014543FC0
:1017C000F57002173BB411DE90D001E054C0F00276
:1017D0001489E56054F0B4200050267A0060027A43
:1017E0003090D001E054C04412121900440812197C
:1017F000001218EE54FD12190044021219000218CA
:1018000087E560B420367A8012189154F7121900D7
:101810007570007F0690D002E0A2E5E57033F570A8
:1018200090D001E0121901DFEC54FD12190090D0A4
:1018300001E054C0F079707E010214C7B421127A1D
:101840003012189154F512190044021219000218AE
:1018500087B422057AFF02186CB423057A000218B7
:101860006CB428004028B450005023FA1218915448
:10187000F51219004402F0800490D001E012190121
:1018800090D002E030E5F290D001E054C0F00214B4
:101890008990D001E054C044131219004408121971
:1018A000000218EEE56054C0704190D001E054C0D1
:1018B0004412121900440812190074404560FA12CB
:1018C00018EEAA611218EEAA621218EE54F5121957
:1018D000004402F0800490D001E012190190D0027F
:1018E000E030E5F290D001E054C0F00214897F08A6
:1018F000EA33FAE054F750024408121900DFF122EB
:10190000F04404F054FBF02290D003C2AFE0441046
:10191000F0D2AFC2DA1214EFE5605001C4540FFFE9
:10192000C2DAC2DBBF0400400CBF0800503DD2DB6E
:10193000EFC39404FFD2D8E5D830E1FB90D003C2C6
:10194000AFE054EFF0D2AFC2DABF0004E5DA8013A3
:10195000BF0104E5DB800CBF0204E5DC8005BF03AA
:101960000AE5DD7970F77E010214C7021489E5608B
:10197000605AB40111E5637F06123317D2C0C2C0AA
:10198000C2C5C2C68046B40211E5637F0812331790
:10199000D2C1C2C1C2C5C2C68032B40311E5637FE1
:1019A00008123317D2C2C2C2C2C5C2C6801EB40456
:1019B0000D1219CFD2C3C2C5C2C3C2C6800EB405B0
:1019C0000B1219CFD2C4C2C5C2C4C2C6021489E563
:1019D00061123537E562123537E563123537C2C516
:1019E0000000C2C600D2C5221214EF5007122E9E6C
:1019F000E4122F5990D001E044C0F01233B990D0D6
:101A000002E020E4071215F570F1802D540FFF124B
:101A100014EF400E901A53EF93FF7414122F6802C4
:101A20001A2A901A43EF93122EC01233B990D002A3
:101A3000E030E4C71215F570F190D001E0543FF0AA
:101A40000214893132334134353642373839432A2A
:101A50003023440102030D0405060E0708090F0B8D
:101A60000A0C1030210CD211C2101233B9125DC70A
:101A700080F11236C6C24EC220E490C0617F04F0ED
:101A8000A3DFFC90BF2DE05407901A8FFF2F7380C7
:101A90000E8010801280148015801880028000D380
:101AA000021AB8C3021AB8D3021AB8C3800A90C087
:101AB000F5800390BF2FE013921890014E30180369
:101AC00090014DE583FD4480F53FAE828E4090C08D
:101AD0006C12315BC21A1233B97E1512357E123385
:101AE000B975390078BD764B78BDE6603312204574
:101AF000402812375960F175390178C1767D12336B
:101B0000B978C1E6601A121F376405605C204E0D7B
:101B100078C5E6600B12204550E4122461021A6376
:101B20001230B870B9D211C210204EF190BF2CE023
:101B3000601190BF2DE05407600464017002B21878
:101B4000021ABA90BF2DE05407FF600E6401600ACC
:101B5000EF64047002B218021ABA102004D2208076
:101B6000F41230CD60EF021BFAE53B90C06AF0A39F
:101B7000E53CA21892E0F012203A790190BF2CE0E7
:101B8000601790C0F41231431231186003021C1127
:101B900090C0FB123143021C171231EC90C0F412BA
:101BA0003143123118700EE990C0FFF090C0FB1263
:101BB0003143021C1709E990C0FFF0B9060040D973
:101BC0007901E990C0FFF01231EC90BF2DE054078D
:101BD00060046401703B10201CD220853D4B90C0F6
:101BE0006A12314390C06112315BA3E53FF0A3E577
:101BF00040F0021B551230CD6017B21890014E30E4
:101C0000180390014DAD83AE8290C06C12315B80A1
:101C10000690C06C12314390C06E12315B90C0755B
:101C2000E4F0A37401F0A374C2F090C0FAE0A2E45F
:101C3000923DD20C021C37C20F1236C61233B99035
:101C4000C06EE04440F53FA3E0F540C21AAE3D123D
:101C5000357E1233B975391078BD764B78BDE660A4
:101C600034122045402A12375960F1C20B753911E0
:101C700078C1767D1233B9121F3764056021204E7A
:101C80002978C5E6600F78C1E6600A12204550E465
:101C900012246180A21230B8600280B6021B25AD0A
:101CA0003BAE3C12311824FE5003021A6390BF2D44
:101CB000E05407FFB4050B90BF2E123143123118C8
:101CC00070DA90C0F4123143123118C36006EF6429
:101CD0000460C9D39210C21190AEABE030E22D3057
:101CE000102690C0F412314390C06AE06D547FFD1D
:101CF000A3E06EFE90C0FEE0540F600C04FFEE33D4
:101D0000FEED33FD4006DFF6D2068016C206021D48
:101D100022AD3BAE3C12311824FE5006122079024F
:101D20001A6390C049E0A2E39204A2E29203A3E006
:101D3000A2E79201A2E69200A2E0920212203EA344
:101D4000E0A2E79207547F04F53E90C048E0FA30E5
:101D5000E00E90C0531231437F05123172021D6EA6
:101D600090C06C123143200705E53D1230A490C0AD
:101D70007012315B90C049300A08E0132010011343
:101D80004005C205021E24D205EA30E11490C0507D
:101D90001231437F0412317290C075E4F0A3123106
:101DA0005BEA20E203021E2490C04CE0FFA3123144
:101DB0004390C072EF540FF0A312315BC20C12308B
:101DC000FA6003021E1EA3A883A982123143A3E076
:101DD000FF90C074122084402F90C077122084405E
:101DE00027EF9405EE9400ED9400401C88838982CF
:101DF000E05410700D122F82A3122F82A3122F8293
:101E00008006E0540F122F8290C072123143A3E07B
:101E1000FF88838982A3A3122084400880001220B7
:101E2000790220ABEA20E70AE53954F0B420090230
:101E30001E40122079021A6378CF761F78C6760684
:101E40007539201233B9121F37B40203021ECCB405
:101E50000503021D11207D4FE55554BFB40048E530
:101E60005654BFB4004178D2E60866703A90C0F18B
:101E7000E0703478CAB6002F205E2CE55D641360F4
:101E80002630350E78C6B6002112337FC239C245DE
:101E9000801820AA0610450A103902800D1243E06E
:101EA00080081245658003122079204E1378C5E61C
:101EB000600E304F061220790220B378CFE670060C
:101EC000122079021A63021E43021E1E123741605D
:101ED0000EB4402312305E701B753924021E43205D
:101EE000101212305E700D1220727008C20912209A
:101EF000790220A7021E40B480FAE539B424F51215
:101F0000205650F012307C70EB122062601BB40738
:101F100006122079022096B41EDA3006D712206EFF
:101F2000B405D112207902209912207270C6D2090C
:101F300080BC12375C8003123759600B14700F128B
:101F40001F485339F0740122E490C048F022123740
:101F5000414006121F4874022212204AFE4016E534
:101F6000395403901F69020B6C021F78021F78021C
:101F70001FA5021FB5740322BE6028121F48788671
:101F80007D047F0312300A18E60303540FF53A1854
:101F9000E654FEF53C18E6547FF53B74027839D6DA
:101FA000740422E422BE709774037839D67E0090C0
:101FB000C049021FE0BE000890C04C7E04021FE032
:101FC000BE402D7883E6540FFF2F2FFF90200A93F9
:101FD000FE601D20E7140FEF93CF0493F5828F83EB
:101FE0007F037883E6F008A3DFFA90C048E04EF064
:101FF000783A16E6600274FF798667335009E66026
:1020000003740422740522021F3F000000800000B8
:1020100002C04F00000000000000000001C052009C
:10202000000010C05520C05840C05B0000000000F8
:102030000000000000000000000090C04AE00354CF
:102040001F04F53D22A211824F227886E65470B417
:102050001002D322C3227883E65430B43002D32254
:10206000C3227885E61308E6C492E4541F227884DC
:1020700080F290BF6CE0540122203503123399782E
:10208000C6760622E0CFC39FFF1582E0CE9EFE15E6
:1020900082E0CD9DFD22E480077408123031745334
:1020A00078C1F674308006744080027450F539743B
:1020B0003F80067460F539747D78C6F6C219123314
:1020C000B9123330AE3E90C070E04420F53FA3E03B
:1020D000F540C21A12357E122548600540D5022C03
:1020E000DD1233B912255E74FA200202746478BDE1
:1020F000F61233471234B11237596402601478BDB6
:10210000E670F478C6E660071230B8600280C80254
:10211000244012374120020A648060DB123126E439
:10212000801750D312204A50CE1231267885E6A26D
:10213000E3920B18E623C454077852D630740CE6A9
:1021400012343D123759E57F20E5F81233B975474F
:102150000075480A754900754A0AD208300B030217
:1021600023A21224A312375978C5E6602578BAE66F
:10217000084670F112254860084003022CDD022059
:10218000B31233B9123138400C0547E548B5470062
:102190005037022440754700E55212343D12368D07
:1021A00078B9761D30082C123138501178B9E624F0
:1021B000F940F4123138501B78B9E670F612323219
:1021C0000549E54AB5490040C978C6E660C412240D
:1021D000B38092123759301BFAC21B123405E5390D
:1021E000B44000500E12375978C1E670F812302F03
:1021F000022CDDC213C24D78C176D078397404D672
:102200001233B91237596402600D78C9201302786D
:10221000C1E670EC0222FDE539540FB405028014CA
:1022200040030222BF123741B440D512305E700223
:10223000053980CC123741500E12204A40C280BB73
:1022400078397404D680DEB480F6788BE630E10508
:1022500012307C70A60539122056400FE5396456BD
:10226000609920050302237A02230DE539B466380C
:10227000122062B40406122450022CDDB4090612A6
:102280002461022CDDB41D030221FBB40C0F1224C7
:10229000D8C2196002D219E4F546022200541CB4D7
:1022A000141A122D4D022200122062B403030222DE
:1022B000FD7839B656D5B40D0302230D0221FB1269
:1022C00037414015B48017204D2B1224DFE53954D7
:1022D0000FB4060D053902220012204A40F80224EC
:1022E00040E54660F978C6E660F4D21A5339F01238
:1022F000357E0220D712205640E4022262E539548E
:10230000F064506003022440D2D502231BC2D59052
:10231000C06A12314390C06812315B200C521230F7
:10232000FA600C90C06A12314390BF1E12316120D6
:10233000D50B90C075123143A3E0FF8007E4FDFE8A
:1023400012248EFF90C074E02FC0D090BF22122FB5
:102350008290C073D0D0E03EC0D090BF21122F82B7
:1023600090C072D0D0E03D90BF20122F8220D507C0
:10237000E53954F0B45003022CDD1225134020122D
:1023800036D6122DAD1235441236A01254AEE539B0
:1023900054F0B44005D212022710C2120228A20241
:1023A000244078C2763E0539121F376405601078E4
:1023B000C2E6600878C5E670EF022CDD022440E535
:1023C00039B4530EAD3BAE3C12311824FE5003021B
:1023D0002CDD90C048E0FA30E41EE539B463199072
:1023E000C0FDE0540F0490C056B4090040039408A7
:1023F000A3FFE033DFFD5048EA30E50890C059E024
:10240000A2E79208EA30E615E539644390C05C60C3
:1024100001A3E0540FF54AE054F0C4F548E539B49F
:102420005318EA30E21490C04CE0FFA312314390FD
:10243000C072EF540FF0A312315B1224B702216572
:10244000E539B46000400675396F122450022CDD66
:102450005355DF1233B9740912303178C9760680CA
:102460000F5355DF1233B9740A12303178C976062A
:10247000C2541233B9123759304F0F78C9E670F28F
:10248000C24F306505743B125CCF12302F22740AA4
:102490001224D1042274291224D190C08BF022740A
:1024A0007980F474741224D178BAC2AF760008F639
:1024B000D2AF2274FB80EE74051224D104FF74BCE9
:1024C0001224D18FF0A478BAC2AFA6F008F6D2AF2A
:1024D00022858AF0A4E5F0227885E6035407227A63
:1024E00086EAF8C39482FD7F0112300A1A1890C060
:1024F00070123143E6547F6016141230A412252561
:10250000400D794607E729F9EAF8E6547F14F7BA4F
:1025100083CF227885E6547FFD08E6FE7F041231E2
:10252000724DD3600E90ADEBE020E30890029B1259
:102530002540B322900320122540B350F69003DFCC
:10254000C3EE9582ED958322E53954F0B45005A28F
:102550004F500922B46005A24F400122E422E53920
:1025600054F0B4300302263BB440030225E6B450D5
:102570000302260EB4600302257B2212265C75F04E
:1025800088A2101226637B0112269530F10B0B08EE
:10259000080812268E081226B83004050B081226E9
:1025A000C5083055203079061226F20225D6E8FA01
:1025B000785F7F047D10122FF9E55F540F44A0F57A
:1025C0005F055EEAF81226D430550B786E7F047DE5
:1025D0001012300A155E8B33788BEB14C446F6125A
:1025E00038E308DBF52212265C75F080A20912267A
:1025F000637B0112269530F10B0B08080812268E1A
:10260000081226B83004050B081226C580C8122609
:102610005C75F08A122695089026387F03E493F6BD
:1026200008A3DFF91812268E081226B87B023004A0
:10263000050B081226C5809E00368012265C75F0B8
:10264000821226950812267012268E081226B87B52
:10265000023004050B081226C50225D6788B7F2A86
:1026600002301B7203721990AEABE072E392F1225A
:1026700088F078867F037D0312300A7984A8F0E71A
:10268000540FF60809E7F60809E75480F622E6A297
:102690001992E6F622788BA20492F2A6F090C0F787
:1026A000087F04E0F608A3DFFA798C90ADEBE03008
:1026B0007402540CC4D7F72290C0F6E0F608A3E0E9
:1026C00054F0F6082290BEC27F04E0C4D608F6A3F8
:1026D000DFF8082212577F0B600AFE795F7F04E75C
:1026E000C4D6DE012208F609DE0122DFF20B08085B
:1026F00080EB0B90BED1E0FE90BED27F04E0C4D64A
:10270000DE012208F6A3DE0122DFF20B080880EBCF
:1027100075397078C176D01233B9122CFE6402601C
:1027200015122D8B4003022CD178C1E660F81234CB
:102730009B12349580E1122DBB70E6122056500E8C
:10274000122D4E60DC149027719390275873122538
:102750001340CE122D2280B8022CA6125686122DBE
:102760003B02279E80FB122D4302277C02277C80A0
:10277000A90017030C0E17141717171775397712BE
:102780002DC91236B212349B123495122CFE122D22
:102790008B4003022CD1122DC350EA02271078C9B6
:1027A000764778C1761512368075397112349B12CE
:1027B0003495122CFE122D8B4003022CD178C1B619
:1027C00000EA0227C578C97647753971800312334C
:1027D000B9122CFE6402601B78C9E66005122D8BCD
:1027E0004003022CCE304F0302289D12349B12343A
:1027F0009580DB122DBB70E0122056500E122D4E2C
:1028000060D61490283E939028137312251340C865
:1028100002286E1256971236A012302F78C2761503
:10282000022C8512302F1236A0022710122D3B8069
:10283000948092122D43022849022849809000106A
:10284000191E20292629292929753978122DC912FE
:1028500036B212349B123495122CFE122D8B40038B
:10286000022CCE122DC350EA1236800227C978C13D
:1028700076157539791236A01233B912349B123499
:1028800095122CFE122D8B4003022CCE78C1E670DF
:10289000EA122D221236801233B90227C91236A04D
:1028A000D24D1256C7E478C0F678C9F6C24978C24C
:1028B000761578C376D178BD764CC214300F0302FA
:1028C0002C85E555540F6405600B6405640C6005A8
:1028D00074041230317539821233B9122CFE64023D
:1028E000700302294B122D8B4003022CD1304FCFA5
:1028F000304919C249200D14122D0D12347DE49077
:10290000C047F01236BF123680022A1F78C1E67027
:1029100008300D05C20D022974200E27E5554556D5
:1029200020E42620E52320E7206406600B204408ED
:1029300020630512349E800312349B203B0812341E
:1029400098800612349B123495808D200D1E122D16
:10295000BB70191220565017122D4E600F122D0DFC
:10296000122D4E149029F59390298A730228E512AE
:10297000251340F8122D0D12347D122D22123491A0
:1029800012348978C376D10228D8022C850228D83F
:10299000C24F12347D02275BC24F12347D12302F9A
:1029A000022761122D4378C1760012348D022A006D
:1029B00078C376D180F0122D4D80EB78C9E6700394
:1029C0000228D8122DDE12348D78C17600022A0337
:1029D0007408123031745378C3F612348512348D72
:1029E000022B1C740912303174A680EB740A123069
:1029F0003174A680E20003060E1931262C46596276
:102A0000122DC91236B275398512349B122CFE1262
:102A10002D8B4003022CD1122DC350ED0228C27819
:102A2000C1761175398380031233B9122CFE64020A
:102A30006022122D8B4003022CD1304F4378C1E627
:102A4000700A78C9760B1236A00228C212349B1283
:102A5000349580D7200DDB122DBB70D61220565036
:102A60000E122D4E60CC14902B1193902A8073126D
:102A7000251340BED20D78C176151236A00228C2A9
:102A800078C2E660061236A0022C8578C1743A2618
:102A9000F6022CB680951236A0C24F12347D022762
:102AA0005BC24F12347D12302F022761122D437406
:102AB000041230311236A078C1760012348D022A09
:102AC0000080EC122D4D80E778C9E67003022A2BB6
:102AD00074041230311236A0122DDE12348D78C1FA
:102AE0007600022A0378C1760074081230317453DC
:102AF00078C3F61236A012348512348D022B1C7462
:102B00000912303174A680E8740A12303174A6803C
:102B1000DF001416212C484143657F88122DC9120D
:102B200036B275398512349B122CFE122D8B400360
:102B3000022CD1122DC350ED75398480031233B9A4
:102B4000122CFE64027003022BBC122D8B40030278
:102B50002CD178C3E6701212302FE530B42703026F
:102B60002A2378C376D10228C2204F19E530B42732
:102B70000878C2E660061236A0022C8578C1743A45
:102B800026F6022CB6304917C24912347DE4200DD6
:102B90000E90C047F01236BF12368078C176117899
:102BA000C1E67010100D49E5306427700778C976CA
:102BB0000B1236A012349B1234958084200D18120B
:102BC0002DBB70131220565011122D4E6009149017
:102BD0002C7A93902BF673022B4A12251340F8E5BA
:102BE00030B4270CD20D78C176151236A0022B3DD9
:102BF000122D22022B3DE530B4270878C2E660068C
:102C00001236A0022C8578C1743A26F6022CB60240
:102C10002B3D1236A0C24F12347D02275B1236A024
:102C2000C24F12347D0227611236A0122D43123496
:102C30008D022B1C78C9E67003022B3D122DDE128B
:102C4000348D1236A0022B1F1236A080E1122D4DBA
:102C500080DC7408123031745378C3F61236A01237
:102C6000348512348D022B1C740912303174A68005
:102C7000E8740A12303174A680DF00191C27323E36
:102C800052575C727B122D0D75399A1233B9122C82
:102C9000FE122D8B4003022CD178C2E6600812345C
:102CA0009B12349580E8122D0D12302F12347D784E
:102CB000C1764B12368075399B80031233B9122CC2
:102CC000FE78C1E6600B12349B12349580F01256E8
:102CD0009712302F12347D12323212552AE490C0EE
:102CE00047F0123369C263C255C21A204E0D90C01C
:102CF000F5E0652354017003021C37021A63123792
:102D0000A47009307A06E55212343DE422301409E9
:102D1000122D1AC21478C376D122E55212343D0224
:102D200036A0123680743F12374D123232740312BD
:102D3000374D1235441236A0022DAD754E00740782
:102D40000230311224D87852D6E602343D221220C5
:102D500062FE6414541C7F086020902D7F1FEF9347
:102D60006E6017DFF9741E6E701012206EFE902DCB
:102D7000877F03EF936E6004DFF9EF2274082F2240
:102D80000306010A0B080714050201203B29300E37
:102D90000A78C6E67005122DC3401EE5515403643F
:102DA0000C6012E5260303655154037008C20E78C7
:102DB000C676348002D20ED322C3227883E66526FB
:102DC000540C22E530B42D002212265C788B12269A
:102DD00070788BE64490F61238E3753301221226A0
:102DE0005C788BFB1226D4788BE64480F68B33EB31
:102DF00014C42346F61238E308DBF422AD83AE8216
:102E0000228D838E822222222222122E145004121C
:102E10002E25D32278D0E60866600890C078868296
:102E2000E0D322C32278D106B68202767822785E79
:102E3000B620005013F5F0795FE6122E60067F1180
:102E4000122E57E9F404F622F5F0785E741028F893
:102E5000E5F0D6785E80E77900E629F908DFFA2206
:102E6000C31392D529F9E5F0540F20D503C4F722F6
:102E7000D722795F14C31392D529F9E720D501C46D
:102E8000540F22785E7F1202301B90BF6014C31370
:102E900092D52582F582E43583F583E080DE7422C5
:102EA0007F08022F68122FA3022EC0E55C122FB2FA
:102EB000022EC0122FAC022EBC122F9D122F4AEAF6
:102EC000022F52122FA3022EDC122FB2022EDC127E
:102ED0002FAC022ED8122F9D122F4AEA022F4AE55C
:102EE0003F54F0701AE540122FC9FEADF0E53F5493
:102EF0000F78027956122F22ED122ED5EE80BA7E6F
:102F00004333400C7E503340077E413340027E44C1
:102F10007453122EDC7443122EDC744E122EDCEE2F
:102F2000809E600BFFEE29D4FEED38D4FDDFF62243
:102F3000FF74B08033FF7490802EF8E53954F0B4FC
:102F4000F00122E874F080207420FF7410022F68D2
:102F50007420FF7418022F68E4FF90C087F0E480AB
:102F600007FF90C087F07401F5F078D290C0A0867A
:102F700082E5F0F0A3EFF0E62402B4F00274A0F6CC
:102F8000EF22F5F0E065F06010E5F0F07FA8E06575
:102F9000F06006DFF9E5F0D322E5F0C322FA122F44
:102FA000A3CAC4540F2490D43440D422FA122FB2AE
:102FB000CAC4540FB40A00500280E8902FC3C394CF
:102FC0000A9322302A2320205075F00A84AFF0752E
:102FD000F00A84C5F0C44F22FFC4540F75F00AA450
:102FE000CF540F2F22E6122FD8FE18E6122FD875D5
:102FF000F064A42EFEE435F022EF600DEDFEE8F95A
:10300000C3E713F709DEFADFF322EF600DEDFEE808
:10301000F9C3E733F719DEFADFF322E4F608DFFC41
:10302000227F06E6F70809DFFA22E55C640B2274CA
:10303000007855D622540FB41A00500590304493AE
:103040002274002200C0E0D0C4E4D4C2E2D2E6C6BA
:10305000D6F0F4F2F64044424680A090B08890C08A
:10306000F77883E066540F7012A308E066700CA333
:1030700008E0667006A308E06654F02290C0F6E00F
:10308000FDA3E0FE7F021231727883ED66540F706B
:103090000508EE6654FC22C5822440C582C58334EF
:1030A00000C58322780030180478FFF404F9023058
:1030B000B1EE29FEED38FD227845E61846600DE4B4
:1030C000863FF608C6F54012356974012290C06348
:1030D000E0FFA3E04F6022854B3D90C06112314379
:1030E00090C06A12315B90C063E0F53FE4F0A3E06A
:1030F000F540E4F01235697401227F0190BF1E1281
:103100003143A883A982123118898288836008A379
:10311000A3A3A3DFEA74012290C06AE06DA3700349
:10312000E06E227402227883E65430C490313493E6
:10313000788AF622001F637CE53854072402540D78
:1031400024FB22E0FDA3E0FE22E0FDA3E0FEA3E0DD
:10315000FF22E6FD08E6FE08E6FF22EDF0A3EEF012
:1031600022ED122F82A3EE022F82E0FD123097E0B3
:10317000FE22C3ED13FDEE13FEDFF72290319CC259
:103180007CE9600CA2E0927CB27CB406004001E4D1
:1031900025E0FF93CF04938F83F58222A02BA02BF1
:1031A000A2EBA5ABA86BAB2B9031AD80D2A0ABA0AE
:1031B000ABA36BA62BA8EBABAB9031BE80C1A1EB50
:1031C000A1EBA4ABA76BAA2BACEB9031CF80B0A244
:1031D0006BA26BA52BA7EBAAABAD6B9031E0809FE8
:1031E000A2ABA2ABA56BA82BAAEBADAB7C0B90C09E
:1031F000F4122DFC12317CE0FA123097C082C083A9
:10320000122E01EAF0A3122DFCD083D082DCE8223A
:10321000C082C083122E01E0A3122DFCD083D08285
:10322000122F82123097DCE8025C7590D002E0A287
:10323000E6225324F3E5241232DD123405E4C2AF52
:10324000F530C21EC20DD2AF907001F022E53924D4
:10325000D04022E555455654BFB4001978CAB6008F
:10326000051232B38006B6010C1232C7206B1AD297
:103270006BD24780141232D640051232CA80031234
:1032800032C1306B04C26BD24790C067E0652560E5
:1032900005E52512330590C066E065536005E553EA
:1032A0001232F390C065E06524543C6005E52412B9
:1032B00032DD22C2C790D001C2AFE054DFF0D2AFFE
:1032C000221232CAD2C722C2C72290D001C2AFE0B6
:1032D0004420F0D2AF2290D001E0A2E52290C06558
:1032E000F0543C44027F06123317D2C0C2C0C2C59C
:1032F000C2C62290C066F07F08123317D2C1C2C185
:10330000C2C5C2C62290C067F07F08123317D2C26E
:10331000C2C2C2C5C2C62213C2C592C600D2C5DF90
:10332000F622123355D2C3C2C5C2C3C2C6D21D22B1
:1033300090D003C2AFE04408F0D2AF3074057F0BE9
:10334000022F3A22123330123355D2C4C2C5C2C43E
:10335000C2C6D21C22900190E583123537E5821255
:103360003537C2C5D2C6D2C52290D003C2AFE05411
:10337000F7F0D2AFC21C3074057F0C022F3A22C284
:1033800037C235D234907004C2AFE526F0D238C2CD
:10339000AAC2ADD2AF1233B922D237D235A234C2CB
:1033A00034907004C2AFE526F0907000F09238D2ED
:1033B000AAD2ADD2AF1233B922C27F2275F8005320
:1033C000880F20340E758AC0758CB4758BB3758DDB
:1033D000FF800C758AC0758CB4758BB3758DFF75C5
:1033E000890075F8C02243254053257F0233FB53E3
:1033F000253F0233FB5325BF432580E525023305D6
:10340000C2B4D21F22D2B4C21F2290D003C2AFE0F6
:103410004420F0D2AFE57F54107021437F107F0726
:10342000022F3A90D003C2AFE054DFF0D2AFE57F75
:1034300054106008537FEF7F08022F3A22C27A545B
:1034400007FFE420740690ADEBE05403FEC39FEE4B
:103450005001EFFEC47852D6C63074086654F0604E
:1034600003437F20EE307408B275A275E43403FE86
:1034700090D003C2AFE054F84EF0D2AF22432506FD
:10348000E525023305D22A80F7C22A80F3D22980AB
:10349000EFC22980EBD22A22C22A22D22922C229B3
:1034A0002274000232F31232F3432430E524023254
:1034B000DD301C26E5402485FEE53F540F34003006
:1034C000E207FDEE2401FEE43D5403FD906AE7129D
:1034D0003513D2C4C2C5C2C4C2C622E5402485FE8B
:1034E000E53F540F340030E207FDEE2401FEE43DD9
:1034F0005403FD9065EF123513D2C3C2C5C2C3C2D7
:10350000C6301C0E906AE7123513D2C4C2C5C2C4BD
:10351000C2C622EE2582F582ED3583F583E43400C0
:10352000123537E583123537E582123537C2C500CB
:1035300000C2C600D2C5227F0833C2C592C600D2DF
:10354000C5DFF62278867D037F0412300A18864094
:1035500018E65407F53FE623C454077952D7E7121B
:10356000343D7883E6C41236E61234DB7433123706
:103570004D12372E22E546600302360BD32278D84F
:103580007600087600F544F545F542F543201AE546
:103590008E461234DB74331233B912374D1236446F
:1035A000F57B741A12374D123644B57B004002F594
:1035B0007B78D8E6B57B005013A67B08F68542449D
:1035C000854345853F428540430235DC78D9E6B5E1
:1035D0007B005008A67B853F44854045784616E62B
:1035E000603D201A2620180FE5402401F540E53FF4
:1035F0003400F53F023604E540C39401F540E53F51
:103600009400F53F1234DB741A808C7846E628F873
:10361000E612362E540F4410F53F8E400235925379
:10362000420353440385423F8543400235697D0090
:10363000301804F4047DFFFE90C071E02EFE158268
:10364000E03DFD2290D003C2AFE04410F0D2AFC203
:10365000DAC2DBD2D8E5D830E1FB90D003C2AFE0CC
:1036600054EFF0D2AFE5DA22E6247AF618E6340316
:1036700030E209F608E62401F618E4365403F6228F
:10368000D222E5241232DDD21E75302722D222C288
:1036900023E5241232DD123400537ADF7530032221
:1036A000D223C222E5241232DD123400C21E75304C
:1036B0002A22D222C223E5241232DD75302D22C205
:1036C00024E5240232DD907004C2AF432603E526D0
:1036D000F0C23ED2AF22907004C2AF5326FCE52662
:1036E000F0D23ED2AF222323540CFF9070047826F0
:1036F00074F3C2AF564FF6F0D223D2AFE5240232B4
:10370000DDC223E5240232DDD22322C22322C228D5
:10371000E525023305D228E525023305C4035438D4
:10372000C2AF5325C74225E525D2AF023305E47861
:1037300080C2AFF537F536F6C23CC23BC23FD2AFCE
:10374000227883E654C0B4C002D322C32278B9F6EB
:10375000125DC778B9E670F822125DC71237736040
:103760001114600E12382512390CB40203740122B0
:10377000740222E4303C29123801701178C57603B6
:10378000E4F537203B1BC23CD23B02379E303B075F
:1037900005377405B5370AE478C5F612372E74017B
:1037A00022740222125DC71237C660191460161205
:1037B000387812390CB402037401227883E654C0BD
:1037C000B480F5740222303B1F203F2A7402203C53
:1037D0001678BEE6701012372E907004C2AF5326D2
:1037E000FCE526F0D2AFE422907004C2AF303FEE89
:1037F000D2AF78BE7618C2AFC23FD23BD2AF74010F
:10380000227882E6FD18E6FE18E6AF35BF00030217
:10381000381BCD33CE33CECD33DFF754076407707A
:1038200003EE641222E5347823C398400278007FC7
:103830000712389EE535045407303D02240404FF86
:1038400078897D0712300A18E654E0F918E6541F0B
:1038500049C403C6F5F018E6A2F633A2F533C6F55F
:10386000F03318E6131313C4A2F61323C618E63375
:1038700033330303C6C23C2290C0007D05E0F4242C
:1038800009FFA8820888827E06C3E013F00582DE65
:10389000F9DFF2DDE87F05780212389E80D7798360
:1038A00090C000800209088882E0FA74072582F53A
:1038B00082E0FB74072582F582E0FC74072582F51F
:1038C00082E0FD74072582F582E0FE6AFAEE6BFB6A
:1038D000EE6CFCEE6DFD4C5A5BCA4B5C5D4A6EF7BC
:1038E000DFC322E4FA7F2466CA08667E10C333CAA7
:1038F0003350066453CA6490CACADF0A18CAC4D6D1
:1039000008F6EAC4D622DEE508CA80DB7A0C7B0022
:1039100012393260130B90395003FF93CF04936038
:103920000ECF2483F8EF66F67A5C12393260010B11
:10393000EB2278837E04E47F086625E050016ADF8D
:10394000F908DEF36625E050016A25E050016A229D
:103950000000040104020440040403100480010474
:10396000040800010320000803010000010802040C
:1039700004100101000202010340000000100000D9
:1039800003020000000000400110000002080000D7
:10399000042000000102030800040180020200006C
:1039A00003800280000000000020000000000000F2
:1039B00003040000000001400000024000800000FD
:1039C00001200000000002200210000000000000A2
:1039D000C0E0C0D0C083C082C2D3D2D4907000F007
:1039E000E5309039E673023A4C023A55023A6102E8
:1039F0003A6F023A86023A90023A90023A90023ABC
:103A000090023AB1023ADE023AE5023AEA023A4C50
:103A1000023A4C023AFB023B08023B1B023A90027C
:103A20003B1B023A90023B1B023A90023B1B023ABC
:103A300090023B1B023B32023ADE023B52023B5CED
:103A4000023B67023B6D023B70023B879070017442
:103A500000F0023BACE5302403F53075320D023B3B
:103A6000ACD53208E4F531F532023AA8023BAC900D
:103A70003B9B7831E693907001F006B60505760021
:103A800075300C023BAC788A907001E6F0023AA8DF
:103A90007931E7248BF8E6907001F007783206B6AA
:103AA000060C7600E724FAF7E5302403F530023BF4
:103AB000AC7931E7248BF8E6907001F00778320694
:103AC000B606187600D53310E57A30E5DB77007559
:103AD0003305753009023BAC75300F023BAC90707A
:103AE00001E4F080C35324F380BE783206B61F0889
:103AF000753000D21B5324F3023BAC90700174AAC2
:103B0000F0E4F531F53280A090700174AAF07832BB
:103B100006B6070476008090023BAC903BA078325A
:103B2000E693907001F006B606057600023AA80208
:103B30003BAC7931E7248BF8E6907001F0077832DE
:103B400006B6060B7600D53303023AA87530330269
:103B50003BACC222D22375302A023BAC90C000E0BD
:103B6000907001F0023BAC753205023A55023A61A1
:103B7000903BA67832E693907001F006B606057683
:103B800000023AA8023BAC7931E7248BF8E690704A
:103B900001F007B70A027700023BACAAAAAAAB89D8
:103BA000AAAAAAAAAF12FFFFFFF550ED78BA79BB17
:103BB000E746600517B7FF011618E66001160243D5
:103BC0006D109803023C06C0E0C0D0E9C0E0C0839D
:103BD000C082E599307324F990BF71E0B4500DB9FB
:103BE00034057935023BECB935027934E979D09066
:103BF000C078878207B782027778F0D082D083D0EE
:103C0000E0F9D0D0D0E010990032C2CF303803C2F2
:103C10003832C291C0E0C0D0C083C082C2D3D2D4F7
:103C2000307D3078D6E6A292B333F608E633F65408
:103C3000F0B4100F18E620E00A79B7E4C6F70809D7
:103C4000E4C6F7C310400A78D5E633F618E633F633
:103C5000B39290E54F2403C54F903C5D73023CBD89
:103C600002427302428F023CBD0242A7023D38026B
:103C70004273023D27023CBD02427D023DB6024234
:103C80007302423E023CBD0242DD023D38024273F5
:103C9000024244023CBD02424A0241FE0242730219
:103CA0003DC1023CBD0240FD023D3802427302416B
:103CB000C7023CBD023CB7123CC0754F0002436BCB
:103CC00020413A10434D104735E57F10E54B78D23F
:103CD000E60866602890C0A086820606B6F00276E6
:103CE000A0E0FF0582E0307D0978D5F618CFF6D246
:103CF00040CF30730878DDF6CFF599D24122E4A2A7
:103D00006B92E0A26C92E1A26D92E2A26A92E37FD2
:103D1000B080D37F80E55780CD537FDFE552C45418
:103D20000744107FF080BF123D2D02436B1041020B
:103D3000800578DDE6F5992278B8E610E402804047
:103D4000F6540E903D4773800E802A803380318078
:103D500032802D802B8051E61318E613B411030234
:103D60003D80FF78D090C078868206B68202767851
:103D7000EFF002436B306908E61318E61378EFF6AC
:103D800002436B3069FAE61318E613A2E0727492EC
:103D900074A2E172779277540CA2E292E4A2E392C9
:103DA000E578DB46F602436BE53954F0B4F0D1E632
:103DB0001318E61380AC10440280031240F502434E
:103DC0006B784D06E55620E50920E70920E4090255
:103DD0003F3A023EA7023EFD30E603023E9AE5541A
:103DE000543FB41A005029123037F553E554A2E776
:103DF000B05292D572E67263A04C9229A2D5824C41
:103E0000922490BF33E0A2E7B39225D22A02436BFB
:103E1000B41A08B60A00505E023E7CB41B07B61EF8
:103E20000050538012B41C1CB632005049B6280012
:103E3000500FB61E005042B614005005B60A00508E
:103E4000380240E4B41D24B66200502AB65D00502A
:103E500017B658005023B65300500DB64E005019F7
:103E6000B64900501A023E79023E86B41E08B60AD0
:103E7000005003023E8D5355EF023F770240E4D2DB
:103E80002574A0023E91C22574A0023E91C2257401
:103E9000B0F553D224D22902436BB62D00400276EE
:103EA0000012401102436B90C047E0C31392D52427
:103EB0005FF9E720D501C4540FB40F0CB67D005054
:103EC00011D229C22A023F77B607004025B60A0060
:103ED00040F37600E004F0F4FF1582E02F400C532D
:103EE00055DF90C047E4F090C046F0D229D22A02B4
:103EF000436B123035F553D229D3023DFE90C047B3
:103F0000B607004018B60A00406D7600E004F0F4F1
:103F1000FF1582E02F400353557F02436BE0C3132C
:103F200092D52449F582E010D501C4123035F553FD
:103F3000432430D229D22A02436B540F903F43FFCF
:103F40002F2F73023F73023F7D023F8B023F93028C
:103F50003F73023F97023FD4023FDC02408C024095
:103F60009A0240AE023F7A0240BF023F7A0240C24C
:103F7000023F7AEAC2E7FA1240F502436BB60B0041
:103F8000400612302F02436B0240E474C41240EE2C
:103F900002436B744080F690C047B60700401AB6E3
:103FA0000A0040D37600E004F0F4FF1582E02F40D1
:103FB00005740412303102436BE0C31392D52449D7
:103FC000F582E010D501C4123035F553432430D2C8
:103FD0002902436BB60B0050D80240E4B62B0040D8
:103FE00014B6A8005008B62C03437F0280857600E3
:103FF000054E02436BB60103437F0112401130624C
:104000000D20770AE54E24FB4004EAD2E7FA02438A
:104010006B90BF31E020E71C90BF36E05403904026
:10402000889390402673E620E00A74CE302E027406
:10403000C40240EE0240F5E6137488302E0274800C
:1040400050077446302E0274440240EE302E09E6CA
:1040500020E0E174880240EEE61424F450CC24FD04
:1040600050E024F450C424FD50D824F450BC80D235
:10407000E61424F450B424FD50BA24F450AC24FDCA
:1040800050B224F450A480AC0011264AB65500501A
:1040900015E630E01174C4023F8DB61500500AB623
:1040A0000B0074C440F1023F77760002436BB615F3
:1040B0000050F6B60B00748040027444023F8D023B
:1040C0003F77301114B60500401AB60A0040D7B643
:1040D0000F004010B6140040CDB619004006123053
:1040E0002F023F7774B01240EED22902436BF55392
:1040F000C224D225227400F5535324CF22E555C59E
:1041000056655654BF6008D2441240F5754D00E51F
:104110005620E67520E51120E70B20E408255654CB
:104120001E90412B7302419C02419F806A8038801F
:104130006B8018805880308012804E804C802880A0
:104140002680438074803F8053803B307019740315
:10415000FFE53954F064F0600BC22FA217727BB3F5
:104160008268922EEF80157401D3FFE53954F06414
:10417000F06008922FA268B07B922EEF655754072B
:1041800060046257D24302436B740280DC302EBE5F
:104190002070BB740080D2C3740480CED380F990A9
:1041A000C047E0C31392D5245FF9E720D501C4547A
:1041B0000FB40F028095D380DF78DBE630E28C20ED
:1041C0007B89D3740580A37857E626540E9041EE80
:1041D000FF93CF0493F5828F83E06654B8600C663A
:1041E000F6F454385325C74225D24302436BBF30FF
:1041F000BF30BF31BF32BF33BF30BF30BF30E53912
:1042000054F064F0601690AEABE030E01FEA20E7B7
:104210000EE57F30E706537F7F437F0802436BE55F
:104220007F20E706437F80437F0480F0E556543FBC
:10423000B40007EA547F70E780D77A1E80E112430A
:104240007602436B1243BE02436B787C90D002E04F
:10425000B60400500C30E416B60302D26F060243D7
:104260006B30E405760402436BB6070040EF76003E
:1042700002436B78BC7F0412428702436B78C07F95
:104280000512428702436BE660011608DFF92290AF
:10429000C089E02424D4F0500BA3E04480F0EA5419
:1042A0007F60011A02436B90C08AE030E72C2481C2
:1042B000B40A01E4F07014D24B90C08BE02410D407
:1042C000F0500678CFE6600116800FB40202D24AA1
:1042D000B40502D24AB40802D24A02436BE55054F4
:1042E00003239042E6738006800B800E804178C5E0
:1042F0007F04124287055002436BE5ED30E41C90C9
:104300007006E0FF907005E0BF04102489500C2473
:10431000FA500D24FA500E24FA500F75510380D52F
:1043200075510080D075510180CB75510280C6E572
:1043300050543C0390433873802A8010801D800EB7
:1043400080228020801E8015801A801A80A7207EFF
:1043500008207F05D27F1233BC809A809878C97F6D
:1043600006124287808F755000808CD291D082D007
:1043700083D0D0D0E032E53954F0B4F0030243BD2D
:10438000E5EDA2E790C060E033F054FF6020B4FF99
:104390002C207B17D27BC216D217D270C27DC26886
:1043A00078EE7607307404C274D27A0243BD307B53
:1043B0000CC216D217D270C27B78EE760122E5EDE0
:1043C000A2E690C05FE033F0B4FF030243D4700F65
:1043D00010720622207208D27278DBE6D2E7F6224B
:1043E000303803C23822C0D0C2D3D2D4C291307D7B
:1043F00038304009C24000000000D3800978D5E67B
:1044000033F618E633F6B3929078D6E6A292B33339
:10441000F608E633F654F0B4100F18E620E00A79F7
:10442000B7E4C6F70809E4C6F7E54F2403C54F9083
:10443000443373024493024493024493024493022C
:10444000449302449C0244930244960244930244DF
:1044500093024493024493024554024493024493CA
:1044600002449C02449302455A024493024493023C
:10447000451C024493024493024493024493024431
:104480009C02449302449302449302448D123CC024
:10449000754F00024560123D2D02456078B8E61068
:1044A000E4028067F6540E9044AB73800E8029803E
:1044B0005A80588031805480528053E61318E61396
:1044C000B411028046FF78D090C078868206B6820A
:1044D000027678EFF002450B306930E61318E613E8
:1044E00078EFF602450B306922E61318E613A2E0D6
:1044F00072749274A2E172779277540CA2E292E401
:10450000A2E392E578DB46F602450B024560E53909
:1045100054F0B4F0F6E61318E61380A990AEABE0C1
:1045200030E01FEA20E70EE57F30E706537F7F4348
:104530007F08024560E57F20E706437F80437F04D4
:1045400080F0E556543FB40007EA547F70E780D707
:104550007A1E80E11243760245601243BE02456036
:10456000D291D0D022C0D0C2D3D2D490C089E0247E
:1045700024D4F0500BA3E04480F0EA547F60011A89
:1045800090C08AE030E72C2481B40A01E4F0701472
:10459000D24B90C08BE02410D4F0500678CFE66068
:1045A0000116800FB402020000B40502D24AB4081A
:1045B000020000E5505403B40340E550543C03901E
:1045C00045C37380158010802A800F802680248048
:1045D000098019801E801E024604207E0C207F095F
:1045E000D27FC2AF1233BCD2AF02460478C97F0675
:1045F000124287800F755000800CB4000778C57F89
:10460000041242870550D0D022C0D0D2D3C2D4FFEA
:10461000E536904616730246880246B10246B80255
:10462000472802473302473E02474A02475602479D
:104630006202476E02478C0247CC02478C0247CC8D
:1046400002478C0247CC02478C0247CC02478C02BF
:1046500047D10247D60247ED02481A0247CC02472B
:104660008C0247CC02478C0247CC02478C0247CCD5
:1046700002478C0247CC02478C0247D60247ED0224
:10468000482202484302484FEF2F543CFD90487F98
:10469000935FFE78800DED936E70130DED93FEE643
:1046A000F45E700A0DED93F536EFF602486EE48085
:1046B000F67D007E800246C17D017E40EF54807011
:1046C000C7D23FE57A20E44E203E1D203D0B7534D5
:1046D000017A0175361E0246E17534007A0075369E
:1046E000458D35EEFB02486E753669753400303BFA
:1046F0000ABA230040107A2402486E7A0043260347
:10470000E526907004F090C0008A820A0AEDF00558
:1047100082EFF002486E90C000EFF07534017A012C
:104720008D3575366F02486E7D027E20EF54C06471
:1047300080808C7D037E10EF54E0644080817D0496
:104740007E08EF54F064200246BF7D057E04EF54DE
:10475000F864900246BF7D067E02EF54FC64480276
:1047600046BF7D077E01EF54FE64240246BF90C021
:1047700000853482EFF005347A0175361E15355305
:104780003507D23C7882EFF6EB0247B090C0008547
:104790003482EFF00534EA24FA7020FAE536240377
:1047A000F536EB0320E7170320E7170320E714FB98
:1047B0005F24FFE53833F53802486E0A80E40320B1
:1047C000E70603F4FB02486EEBF480E3EA24FD8085
:1047D000C8EA24FC80C3EB20E7067880EFF680BCB3
:1047E00023FBE53624DFF53674100247FEE5362458
:1047F000DCF536EBC4FE540F600FEEF4CBF45F240F
:10480000FFE53833F53802480BEEFB7881EFF6E52B
:104810003424BA7002F53402486E7A0075364502C7
:10482000477DE5340534B4050F7880EFF675360022
:10483000BA2302D23C02486E90C0008A820AEFF08E
:1048400002486E7807D8FE90C000EFF002486E79FB
:104850003490C0008782EFF0070ABA0B0E7A01B7D6
:10486000150790C000EFF07701D23C02486ED239B4
:10487000DC047C1ED245D0D0D082D083D0E0320080
:10488000FF0000FFE2000CFFC4010900FF0000FF71
:1048900089030600FF000000FF00000F0E00187FD4
:1048A00071000FFF12070300FF000000FF00003F30
:1048B00038001200FF00001F1C00150F0E001830FA
:1048C0005F08C25F125106124E4E124A9EE55CF618
:1048D000742D122F520570E570B4060022305F0867
:1048E000C25F125106124E4E742D122F527F08785D
:1048F000727971123023A75C057090BF5FE065701C
:104900002278727900E660070908B9080040F6E9E4
:1049100022124A97EFF622E571F9024E60125A947C
:104920007C10125A4FDCFBC322E555540F64002261
:10493000E53954F0648022E55CB40B002290BF4C52
:1049400002494690BF3DAB83AC8290C0FFE060015E
:10495000148C828B8375F003A42582F58222535533
:10496000BF22435510435540227570007F0978716E
:1049700002301B90C098E47F08F0A3DFFC22E55EC4
:10498000B40200401D155E13790F400379F0142422
:104990005FF8E659F6785E122E3E122F58747F02A9
:1049A0002F52D25F125D5E20522E30640302656684
:1049B0002046337403122F617A0790BEAFE0700275
:1049C0007420122DFC122F4A122E01125A4FDAEDCA
:1049D000E070027420022F52755D1A755A04755BDF
:1049E00000D2670250D990BEB9E0540360C5B4024A
:1049F00003024F3B24A3022F59122E9E022F58125E
:104A000049F9E55EFE602B75F00120600330481621
:104A100030590E90C05EE0F5F0E55EC395F0FE05FE
:104A2000F01251AF500DABF0EB122E72122EC90BDB
:104A3000DEF62230481220600F90C05EE0CEC39EAA
:104A4000FCE0FE124A26ECFE744E122F4ADEF922DA
:104A50001249F9E55EC3940AFB7E0B2060033048DF
:104A6000C71251AF40C280CB7871790390AF2B123F
:104A70003097E6C408D6F6E066700912309708D978
:104A8000F1C2D522D2D522124D64E57015702212E2
:104A90004D64E571157122E5717872024AA2E570E4
:104AA000787128F8E622E55CF55453547F4354406E
:104AB0005355BF43551022E55CB40D0040E87452D5
:104AC00080E6745980E2745A80DE745B80DA741E6A
:104AD00080D6741D80D2F5544355104354802274FF
:104AE0005680C5E55CB40D0050D4E555540FB404B0
:104AF000028003B40CB0855C5443551043548022AB
:104B0000E555540FB404028003B40C20785EE660CF
:104B10001B305608C25612577F044001E490C0472C
:104B2000F090C046E55EF0435520D322C322E55500
:104B3000540FB404028003B40C46785EE660413042
:104B40005608C25612577F044001E490C047F078DF
:104B50005F7F047D10122FF9E55F540F44A0F55FCD
:104B6000055E90C049785F7C10124B8390C046E58B
:104B70005EF0786E7F047D1012300A155E4355801A
:104B8000C27822E6F008A3DAFA22E6122F8208128F
:104B90005A4FDCF622305537304C347A0890BEC775
:104BA000122DFC90C049AC83AB82122E01E0A312FF
:104BB0002DFC8C838B82F0A3AC83AB82DAECE49087
:104BC000C047F0124BD090C046F0435580C25522EA
:104BD00090BEC77A087800E0600908540F600408A6
:104BE000A3DAF4E8227F1090C049E6F008A3DFFAC8
:104BF000225355EF53547F5354BF22124AC2742F8D
:104C0000122F59125CCD024C17124AB7024C14C233
:104C10005E124AC212511A125CB8755D00755A00D4
:104C2000755B006003755D18C267C264C2263052AE
:104C300002D26722F57EE57E7F11785E122E577FC5
:104C4000087872022E591250CF90C0F6E0543FFD02
:104C5000A3E0FE7F041231727870124CB490C0F75A
:104C6000E0540FFDA3E0FE7F021231727873124C04
:104C7000B4E0FDA3E0FE7F02124D77ED540FB40BBC
:104C8000004001E4F576E0543FFDA3E0FE7F04120E
:104C900031727877124CB479707E06E7122EC9090A
:104CA000DEF9742D122F4A7E03E7122EC909DEF9B0
:104CB000E7022EAD79007A00ED30E10479057A0C37
:104CC00030E008740229F974382AFAEE75F0648429
:104CD00029F97464C5F02A842904B40B004001E466
:104CE000F608740AC5F08404B40B004001E4F60829
:104CF000C5F004B40B004001E4F622E55DB41A06E9
:104D000090BF2E024D12B4100690C06A024D129050
:104D1000C0F41231437C107B277870124D50EFF6AF
:104D2000087CE87B03124D50EFF6087C647B001290
:104D30004D50EFF6087C0A7B00124D50EFF608EE5E
:104D4000F62290C0FBE0540FFDA3E0FE787080D106
:104D50007F00C3EE9CFEED9BFD0F50F6EE2CFEEDAA
:104D60003BFD1F226009FFEE29FEED38FDDFF82232
:104D7000E6F71819DFFA22C3EE33FEED33FDDFF755
:104D80002290C083123149EDB40A01E475F064A4A5
:104D9000ADF0CEB40A01E475F00AA42ECD3400CFF4
:104DA000B40A01E42DCF3400CF2290C084123143E5
:104DB000EDB40A01E475F00AA4CEB40A01E42E228F
:104DC000125A94402D75F0007E107F00E0600B2F8A
:104DD000FFE0540F600205F005F0125A4FDEEDE5DA
:104DE000F02FFF7E09E02FFF125A4FDEF8EF70021E
:104DF000C322D322155EE57E125A9440F57E20E050
:104E0000F9EE1392D1E920D101C4540F6003122EA0
:104E10002E30D103125A4FDEE6C2D1025A2B7872DD
:104E200090C0987F08E6F008A3DFFA22787290C05D
:104E3000987F08E0F608A3DFFA2290BEDA7A05022E
:104E400007237900801A7903801679048012790883
:104E5000800E7909800A790A8006790B8002790D23
:104E60007F097422122F68E9FF7421022F687401F0
:104E7000022F597482122F5990BEDAE0601B7E090E
:104E8000790190BEDAE9122E8D122EC909DEF39057
:104E9000BEDAE9122E8D022EAD227488022F5974CB
:104EA00089022F59122DFC024EB0122DFC124E6EAB
:104EB000124E607900122E01E993122F4A09DAF599
:104EC00022748C022F59748E122F61900018E49373
:104ED000122ED5900019E493122ED5122F4890BFB0
:104EE00071E0022EB9748F122F617905124E609015
:104EF000BEC2E0122FC9FDC5F0122EC3ED122ED591
:104F00001204E97C037976E7122ECF09DCF9E70277
:104F10002EB37491022F597492022F597493122F49
:104F200061124E5E7469022F527494122F617E07D3
:104F30001251D9E770027420022F52742D122F6182
:104F4000904F5279087A04124EA4122F5074A50281
:104F50005CBF4D6F6465749F122F6179047A0B906A
:104F60004F6F124EA4746F122F5274B1025CBF23A4
:104F7000507267416C70682B53746F7472122F619A
:104F8000904F9779007A0C122DFC124EB5742B12AB
:104F90002F5274B2025CBF4E616D655372636841FB
:104FA0006C70682B7477122F61904FBD79007A076F
:104FB000124EA47444122F5274B3025CBF4368654E
:104FC000636B53504474B4122F61904FD979007AB7
:104FD0000F124EA47466022F52506C732E547572C9
:104FE0006E506F7765724F6666749E122F61905097
:104FF0000279007A11124EA47465122F5274BF0206
:105000005CBF446174614D6F646574C1122F61901F
:10501000501C79007A0C124EA4022F50416E737707
:1050200065724F6E52696E677491122F6190504194
:1050300079017A06124EA47423122F5274CB025CAB
:10504000BF6F2E5365632E23749E122F61905061A3
:1050500079007A07124EA47472122F5274CC025C3B
:10506000BF546F20436C65617274CE122F6179005A
:105070007A0C90507B124EA4022F5053616D652024
:105080004173204C6F632E20202020749E122F61CC
:105090009050A479007A07124EA47465122F5274AE
:1050A000CF025CBF546F2045726173657411022F8B
:1050B000597412022F597413022F597414022F5964
:1050C0007415022F597416022F597417022F597430
:1050D00021022F597428022F597439022F59743A1A
:1050E000022F59743B022F59743E022F59743F020C
:1050F0002F597456022F59746D022F597470022F54
:10510000597471022F59748A022F5974A7022F59AA
:1051100074C9022F5974CA022F59C258E55E700330
:105120000249A42060061249FF022F5890BF73E085
:1051300054032390513773800480278046D258123D
:1051400051974006124A5002514D1249FF1249012F
:105150006068124E427E071251D9E7700274200235
:105160002F52124901700D742B122F597400125CCA
:10517000BF0251E71249F9124E4E1251B5124E427A
:105180000251E71251974006124A500251911249BA
:10519000FF124E420251E7E55E30590990C05EE0D1
:1051A000F8E55EC398B40B0022122F48DEFB22E51F
:1051B0007EB4BE0022124901701DC258740090C016
:1051C00087F09051CF79007A07124EA4022F504EEB
:1051D0006F204E616D65207E087972E77002742041
:1051E000122F4A09DEF522E57E122FC9FAE5F012E8
:1051F0002EC3EA122ED5743A022F52E42011163033
:10520000101390C0F5E0652354017009D2E6201810
:1052100004C2E6D2E7A21092E0A21192E1A24F925C
:10522000E2A24692E3A26792E4A26492E57858C6AD
:1052300066604930E13E125CB8702D20642A125C31
:10524000C4600FB43303025252B43403025252B456
:105250000316E55DB40011E558A2E1743334001281
:105260002F59125CCD1257DB90BF5BE030E0057424
:105270000E123031E558FF7440122F68E4201116E9
:1052800030101390C0F5E0652354016009D2E62088
:105290001804C2E6D2E7A22692E57859C6666007EE
:1052A000E6FF7450122F6822104A1312364490C041
:1052B00095F090C096E025DC1390C096F02290C047
:1052C00095E07F00B4500040190FB4590040130F0F
:1052D000B46500400D0FB4760040070FB48D004058
:1052E000010F90C0F3E06F6007EFF074A0022F6829
:1052F0002290C08DE010E10122F078CEE6703D787A
:10530000CBE6703890C096E0304C05B48D00800339
:10531000B4920050277606E55DB4000A125CC464BE
:10532000186019125337E55554BFB400028003B416
:10533000040A745A024AA87418022F5922227401CE
:105340007F0312535774027F0412535774047F096A
:1053500012535774087F0A557F6006F4527F022F5C
:105360003A22E539B47000401220720E304609909E
:10537000BEB9E0B402005012C24F223046FC90BECB
:10538000B9E0B4020040F32072F078DBE630E7EADF
:10539000C2E7F67D467E5090C09302315B304628CE
:1053A00090BEB9E0B40200401F90C08DE030E2181A
:1053B000C2E2F090C093123143EE4D600C1EBEFF6E
:1053C000011D90C09302315B22E539B4700050F8A2
:1053D000E57F5410600E537FEF7F08122F3A7D0057
:1053E0007E0580DE023423304679E539B471747865
:1053F000C990BEBAE090546393C396406690BEB91C
:10540000E0B4023990BEB7E0B409005056C26DD284
:105410006A1257EE700890BF74E0A2E1926AD24718
:10542000C253C254D24FD23AD263124AD2D25F127E
:105430005CB87006124E2C024C14024C285024C248
:105440006DD26A1257EE700890BF74E0A2E1926AC2
:10545000D247C253D24FD254D25F124AC6124E2CF8
:10546000024C142244403C38104B012290C08DE085
:105470004407F090C08CE02401D4B46001E4F070E3
:105480002C90BF27E02401D4B46001E4122F827075
:105490001C90BF26E02401D4122F821582E0240044
:1054A000D4122F821582E02400D4122F82227F058D
:1054B000122F3A125CB87006124E2C124C14C251C4
:1054C000E4125CDB90C090F0A3F0A3F090C08DE0FC
:1054D000C2E4F0D24C22304C5090C08DE030E04914
:1054E000C2E04410F090C092E02401D4B46001E422
:1054F000B3F01582E03400D4F01582E03400D4F02B
:1055000090BF37E090C09230E710E0B4500CE55502
:1055100054BFB404057406123031E0540FB40709C7
:10552000307406E552C402343D22C24C1259B0C256
:1055300052C257C2565355DF304F04C24FD25F900C
:10554000C09012565490BF4E12494612566890C0F1
:105550009012565490BF3F12494612566890C09020
:1055600012565490BF3C125668C25E125CC9303A63
:105570001090BEC6E02401D4122F821257A4025507
:10558000D2125CB86006124C170255E3125CC4B428
:105590002D030255D2B43500401EB4370050191205
:1055A00057E5206508125CCDC2670255D2743B12E4
:1055B0005CCF124C280255DA648D601630650B12F0
:1055C00050E3124C28D2670255DA124C1712511AC6
:1055D0008011124C1730650BD267755D1A755A0130
:1055E000755B0020620F30460990BEB9E0B402003E
:1055F000500312342390D001E0443FF0C23AC2512C
:10560000C254C2637F06022F3A124E4E90C0FFE092
:10561000700104122EC9742D022F4A122DFC7B0238
:10562000122E01E00E122ED5DBF6122E01E0022E14
:10563000B9122DFC800A122DFCE00E540F122EC35D
:10564000122E01E00E122ED57427122EDC122E011E
:10565000E0022EB9123149BF0100B3E43ED4FFE4A9
:105660003DD4FEE43400FD22E02FD492D5122F82E7
:105670001582A2D5E03ED492D5122F821582A2D5F2
:10568000E03DD4022F82124969124C17D26DD247E5
:10569000D2537F01022F3A7F02122F3A90BEC6E00A
:1056A0002401D4122F82D25FC26DC253D26A125724
:1056B000EE700890BF74E0A2E1926AD247124C17D4
:1056C000205C030257A42212340A90D001E044C0A7
:1056D000F0E555540FB40C0A125CB8700574A612AC
:1056E0002F5920120C12577F9256302703024ACAB4
:1056F0002230531FD25FC26DC253D26A1257EE706E
:105700000890BF74E0A2E1926AD247125CB87003BD
:1057100012511AC256C2575355DF7F02022F3A2048
:10572000573878CCB6004990C0F1E0604314F012CD
:105730005771A2659257500E12577F90C046F0A342
:10574000E4F043552022E55E602678DBE630E6058E
:10575000740C123031D254D24F22E55520E511C2DB
:105760005778DBE630E605740C123031D254D24F54
:105770002290BF34E0540375F020A478CCF622E5E3
:105780005E601DFF7E00795FE754F064F060100EEC
:10579000DF02800BE7540F640F60040E09DFE9EEAF
:1057A000B55E0022125CB86005742E0257B0742DED
:1057B000122F5990BEC6E0022EB990BF5EE0547E13
:1057C000022F8290BF5EE04401022F8278CA025706
:1057D000D378C776072278C7760A2278C77614224C
:1057E00078C7761F2278C776342278C7E62290BF22
:1057F00072E064FF2212589D79DE7E10E0F7125AA3
:105800004F09DEF8755E00795F7E06E0F7600854A8
:105810000F6002055E055E125A4F09DEEE785E02E9
:105820002E3E7401122F6179DE7E0FE77002742024
:10583000122F4A09DEF5E770027420122F5274CD40
:10584000025CBF78DE7F1002301B90BE74025908E4
:1058500090BE7402592190BE7402596D12589D7EFB
:105860001078DEE6122F82125A4F08DEF67E067896
:105870005FE6122F82125A4F08DEF62212584312A8
:105880005D5E7C00EC12585C0CBC1E0040F67C0493
:1058900090BE74E4122F82125A4FDCF722B41E001D
:1058A000B340129058B6C333F5F093F8E5F0049383
:1058B000F5828883C322BBACBBC3BBDABBF3BC0A93
:1058C000BC21BC3ABC51BC68BC81BC98BCB1BCC852
:1058D000BCDFBCF8BD0FBD26BD3FBD56BD6FBD864C
:1058E000BD9DBDB6BDCDBDE4BDFDBE14BE2DBE4447
:1058F000BE5B75F00884FF6005125A4FDFFB2290F3
:10590000BEEC02590890BF051258F2AFF00FBF0964
:10591000027F01E013DFFD2290BEEC02592190BF0F
:10592000051258F2E0AFF0BF0005D2E0022F82BFAF
:105930000105D2E1022F82BF0205D2E2022F82BF0F
:105940000305D2E3022F82BF0405D2E4022F82BFF7
:105950000505D2E5022F82BF0605D2E6022F82D2CC
:10596000E7022F8290BEEC02596D90BF051258F2EB
:10597000E0AFF0BF0005C2E0022F82BF0105C2E127
:10598000022F82BF0205C2E2022F82BF0305C2E3DB
:10599000022F82BF0405C2E4022F82BF0505C2E5C3
:1059A000022F82BF0605C2E6022F82C2E7022F82C3
:1059B000305255206052E55E604E205F4B205048CB
:1059C00090BEB8E004B405004001E4122F8224C860
:1059D0000259D574C8125A94402F785F7E10E6128F
:1059E0002F824025125A4F08DEF478727E08E612A4
:1059F0002F824015125A4F08DEF4124C36E9F40497
:105A0000F56F122F824002C322D32274C8125A9417
:105A1000403B755E00785F7E10E0F66008540F60D2
:105A200002055E055E125A4F08DEEE75710078724F
:105A30007E08E0F60571125A4F08DEF63059091259
:105A40004C36E9F404025A49E0F56FC322D322A38D
:105A5000E582543EB42A03A380F622757E001249E3
:105A600073124E2C125D5E124C36E9F404F56FE5AC
:105A70007E1259D5057EE57EB4C80040EAB4C9005F
:105A80005011757E007C3290BEECE4122F82125AC7
:105A90004FDCF722B40A005005C2D5025AA9B4BEA1
:105AA0000092D5B4D700B3401D905AC7B4640040EB
:105AB00006C39464905B8FC333F5F093F8E5F0046C
:105AC00093F5828883C322B000B019B034B04DB0D2
:105AD00066B081B09AB0B5B0CEB0E7B102B11BB13B
:105AE00036B14FB168B183B19CB1B7B1D0B1E9B2B1
:105AF00004B21DB238B251B26CB285B29EB2B9B224
:105B0000D2B2EDB306B31FB33AB353B36EB387B398
:105B1000A0B3BBB3D4B3EFB408B421B43CB455B410
:105B200070B489B4A2B4BDB4D6B4F1B50AB523B586
:105B30003EB557B572B58BB5A4B5BFB5D8B5F3B6FC
:105B40000CB625B640B659B674B68DB6A6B6C1B673
:105B5000DAB6F5B70EB727B742B75BB776B78FB7E8
:105B6000A8B7C3B7DCB7F7B810B829B844B85DB860
:105B700078B891B8ACB8C5B8DEB8F9B912B92DB9D2
:105B800046B95FB97AB993B9AEB9C7B9E0B9FBA064
:105B900000A019A034A04DA066A081A09AA0B5A035
:105BA000CEA0E7A102A11BA136A14FA168A183A1AC
:105BB0009CA1B7A1D0A1E9A204A21DA238A251A222
:105BC0006CA285A29EA2B9A2D2A2EDA306A31FA396
:105BD0003AA353A36EA387A3A0A3BBA3D4A3EFA40C
:105BE00008A421A43CA455A470A489A4A2A4BDA483
:105BF000D6A4F1A50AA523A53EA557A572A58BA5F8
:105C0000A4A5BFA5D8A5F3A60CA625A640A659A66F
:105C100074A68DA6A6A6C1A6DAA6F5A70EA727A7E5
:105C200042A75BA776A78FA7A8A7C3A7DCA7F7A85B
:105C300010A829A844A85DA878A891A8ACA8C5A8D0
:105C4000DEA8F9A912A92DA946A95FA97AA993A945
:105C5000AEA9C7A9E0A9FBBA14BA2FBA48BA61BA6B
:105C60007CBA95BAB0BAC9BAE2BAFDBB16BB31BBB1
:105C70004ABB63BB7E90A02B78557F41E028F81289
:105C80003097DFF8E8F404022F8290BED0745512EA
:105C90002F8290BEC778557F08E028F8125A4FDF50
:105CA000F8E8F404022F8290BED97455122F829026
:105CB000BED278557F0680E190BF5EE0540122900D
:105CC000C087F02290C087E022E4025CD17400D249
:105CD0005E90C088F02290C088E02290C0F1F0224F
:105CE00090C084E022743C122F5990C096E0FAE4F0
:105CF000304C33BA9900505E04BA9700505804BA39
:105D00009400505204BA9100504C04BA8F0050468F
:105D100004BA8C00504004BA8A00503A04BA870092
:105D2000503404025D56BA9E00502B04BA9C0050B9
:105D30002504BA9900501F04BA9700501904BA9468
:105D400000501304BA9100500D04BA8F005007049C
:105D5000BA8C00500104C39408F404022F52122E8E
:105D600083022E9E025FED0266BD0267D40267F4D5
:105D70000268D60269B3026A54026A68026B7C0246
:105D80006C41026C8202712802714202715B026CEA
:105D9000DF0270DC0271050271870274B00275B80F
:105DA0000275600278BB0279F90286930277DF02FE
:105DB0007AB00287C1026E28026F2C02969A027591
:105DC000E702635902691A12324D12082A50012261
:105DD0001254681254D612571F1252A81252F112BE
:105DE000539D1251FB12533E1253E7125362124954
:105DF000306003025EE5E55DB41D061296DE025ECC
:105E0000E5106F03025EE512986379DAF7303A4FD6
:105E1000125CB87005E55DB400EA90BEB9E0B4026A
:105E2000E390BEB7E0B4090050DAE760D7B40C03E2
:105E3000025EE5B70B20124ACE755D1D755B001240
:105E40005CB8700BC260125D5E12496912510B782A
:105E5000CD7610D25F22125E39C25FE7022E2EE5A8
:105E60005DB400A0B70B1A124ACE78CD7603755DEB
:105E70001D755B01C260C264125D5E12788F0251B3
:105E80000BB70A6178CDE6605CE55E604AB4010D4F
:105E9000E55FC4540FB40A00503D025EC5B404006F
:105EA0005035FC7A017D007E007F00EA122E72B42C
:105EB0000B005023CFCECD0ADCF1124D87BF001767
:105EC000B4C8005012126B0ED26012511AE57EB4A3
:105ED000BE00400302639012639078CC760A90C0B3
:105EE000F17401F02278D2E60866603E122E14505A
:105EF00024FF543FB417028005B418078000122E07
:105F0000258032B41E028008B41F028003B400054D
:105F1000122E258058E55DB40503025F2AB40603FE
:105F2000025F2AB40703025F2A22122E0A400302EC
:105F3000987EFF543FB4171C6FB44004C21680050E
:105F4000B48029C217307024A21672179270207084
:105F50001B0264C2B418166FB44004D2168005B494
:105F6000800AD217207005D2700264E422B41E03A6
:105F700002649BB41F030264A3B43A03026602B432
:105F80003B030266A1F55CB4000302608B90BF7412
:105F9000E020E007206A04D26AD247E55CB43F0300
:105FA00002608B7F0390C082122DFCA3E0122E01B1
:105FB000F0A3DFF4E55CF0307106B41303025FCEAA
:105FC000C271B40D03025FDCB40E03025FD0C25E87
:105FD000E55DB40007305904C259C260E55DB421E3
:105FE0000040047400F55D905D64020B6C30520952
:105FF000755D1A755A0402894EE55CB40D005003B4
:106000000260DC304C031259B0E55CB43000400C47
:10601000B43C0040030266BC540F2423C3940D908B
:106020006025020B6C02614202637D0266BC02665F
:10603000BC0263DA02642302646502647B02647B4F
:1060400002654B0264C00264E202653702656302C6
:1060500065900266BC02657F02649B0264A30266CF
:10606000BC0265A90265AE0265CE0266BC0265DAB5
:106070000265E60266BC0265E70266BC0266BC0217
:1060800033E60233EF0266020266A190BF74E0308D
:10609000E0081257EE7003206A031257CCC25DC2AB
:1060A0005B124BF1205C03304F0478C87615305EEC
:1060B0002AE55DB406030257E0B407030257E01275
:1060C00057DB125CC4B435004011B437004009B44A
:1060D0005609125CD6B457030257E522C25812493A
:1060E0005E206403124C17122F58305F0CC25FC23F
:1060F00048C256122E831249F9E55CE55EB42000D1
:10610000501CE55CB40E02740F122E2EE55CB40E2A
:1061100002740F122EADC260205224024AE3747F33
:10612000122F4AE55CB40E02740F122E2EE55CB4F9
:106130000E02740F122EADC260205203024AC2C278
:10614000502212495EE539B47117C26DD247C23A86
:10615000124E2C124C14C253D254D24FD25F024A68
:10616000B7B46F097400125CDBC24F80EF54F0B417
:10617000803290BEB9E0B4020A303A07C23AC26334
:10618000D2542220550C20560678C0E6600D22021B
:106190004B00307803024B2E024B957411242AF6E3
:1061A000D24980B8E55E60FA125CC46003026221E5
:1061B000E55EB4030DE55FB49108E560B410030239
:1061C00062BA20605CE55EB404005055B40103027D
:1061D00061F3AC5E7A017F00EA122E72B40B0050BC
:1061E00040CFCECD0ADCF1124D87BF0034B4C800D9
:1061F000026201E55FC4540FB40A063065237400DF
:10620000D3501E126B0E4010E55E600CD26012512E
:106210001AE55E700C026307306503024AC2026A27
:10622000FA2059063060030262BA90BF6EE054074C
:10623000906236020B6C0262A602624502624F0255
:106240006274026290E55EB40C00501F0262A6E523
:106250005EB40B15E55FB41808E560B4AA0D0262E0
:10626000A654F0B4A0050262A6403BC259C260D257
:106270005F024C0FE55EB40804E55F80E44027B49C
:106280000A09E55FB48AE4E56080D6B40BDD80C41A
:10629000E55E640370D5E55FB491D07403122E728D
:1062A000B401C80261A490BF6FE030E00DE55EB4B8
:1062B0000108122E72B40A0280B120481130601A0F
:1062C000305904C259C260E57EB4BE00400C127859
:1062D0008F1250E8755D1F024AB790BF23E0A2609D
:1062E00092E0A24892E1122F82E57E90BF5D122FCC
:1062F0008274CD1259D5D25412577179006004D2EC
:10630000277903E9125CDB306511E55E7006124AFD
:10631000C202615C125738D2578014124AB7E55E48
:10632000600D78DBE630E605740C123031D24FD2C6
:106330005F124BD0B40200401F90BF5BE030E71803
:10634000E55EB40A13026348D255C278C27990BEA2
:10635000D1E06004D278D279221248DD701E7979BA
:106360001278AB700B12788F124E2C124C14808660
:10637000124AC212788F124E2C024C142212495E1D
:10638000204F0A205F07E55E60030260DC124AB717
:1063900090C0F17400F01259B0C252C263C24FC231
:1063A000575355DF1264D3D25F12493060163065FF
:1063B00013D267755D1A755A01755B00125CC47063
:1063C000030250E322124AB790BF5FE06006125703
:1063D000C31250ED024C17029C27124930701374FF
:1063E0000412303190BEB9E0B40307303A04C23A27
:1063F000D254C258125CC4B48D030279E212495ED1
:106400005355DF53557FC260C248124AB7105FC769
:10641000125CC4600612511A02641E12497ED25DDB
:106420000257D112495E124AB7124969124E2C1214
:1064300049016016E55E7006124F29024AC22058D3
:106440000912513D12678602645FE55E700E749C0E
:10645000122F59D25F755D20755B00221250D4D285
:106460005F755D0122C258124E1E12495E124AB774
:106470007419122F59755D05D25F22C2581249292D
:106480007003124AB7125CC464CA60091251151233
:106490005CCD0257D11257D1029CF1207704D277FC
:1064A000D276223077FCC2773046F590BEB9E0B4A0
:1064B000020040EC7D467E5090C09312315B80E03C
:1064C000C270C26CD24790AEABE020E114304F11E5
:1064D000026390E539B464004007B468005002D20A
:1064E0000F22D270D26CD247E53964717027125CEA
:1064F000B87021D24FD25FD254C253C26DD26A1249
:1065000057EE700890BF74E0A2E1926AD247124E33
:106510002C124C142212493070FA90BEB9E0B40229
:10652000F3303AF0C23AD254E55DB41A07E55AB4F2
:10653000020280E0C26322124930700C124AB7B2E4
:10654000633063030250DE220260DCC25812495EEF
:10655000124E1ED267D25F755D1A755A00755B00C8
:106560000287C1124AB77431122F5912788F757190
:1065700000124917D264C226755D11755B0022D2E4
:1065800065124ADF755D1A755A01755B000250E3AA
:10659000124AB7757000D25F7472125CCF755D1AC3
:1065A000755A07755B0902510174010265B07402E6
:1065B000126B0E400F126A89E55E60081249306066
:1065C00009026142124AC2024C14024AB722E57A19
:1065D00020E70122122F580209B178CEE660067535
:1065E0005D16757006222278CEE67006755D15027E
:1065F00065F8755D19755A00755B0012496975700B
:106600000A2278DBE620E66DD2E6F6E539B471665B
:1066100030463790BEB9E0B4035BD24FD25FD23A76
:10662000C254C253C26DD26A1257EE700890BF7442
:10663000E0A2E1926AD247124AC6740C12303112BB
:106640005CB87031124E2C024C14125CB87026D219
:106650004FD25FD254C253C26DD26A1257EE700845
:1066600090BF74E0A2E1926AD247740C12303112EA
:106670004E2C024C142254F0B480FA30460C90BEDA
:10668000B9E0B40205303A0280EBE555540F640CD2
:1066900060E3740C123031125CB870D974A6022F0A
:1066A0005978DBE630E614C2E6F6E53954F0B480FA
:1066B0000AE555540FB40C030263902222E55CB442
:1066C0000B20E55E60142048113060051251AF5078
:1066D0000975700090BF6DE0605ED25F124E2C02B3
:1066E000681E5018124AB7125CC464286008E0643F
:1066F0002960031250D4755D02022EABB40C1D123A
:106700004AB7E55E60D42048D13060051251AF50E1
:10671000C97498122F5975700002678BB411141246
:106720005CC4B48D030279E2306005E57E126B0E25
:10673000024C09024C0F0570E570B4BE0050339056
:10674000BF6DE07095E57012590540EAE570E5709F
:10675000124C34E9F404F56FE5701259D55005C2B6
:106760006002681E85707ED260124AB712518302A1
:106770006891757000305FC0124AC6755D01742A59
:10678000122F591257D67428025CCFE570125905A2
:1067900040140570E570B4BE0040F0124969124E15
:1067A0002C7428022F59E570125A94E55EC31334F5
:1067B00000B41000500104FE785FE06670D4081247
:1067C0005A4FDEF6125069E5701251E9124969120A
:1067D0004E2C80B21249375009122EAB755D030260
:1067E0004AB7B4110C125CC4B48D030279E2024CB6
:1067F00009024C0F124937400FB411F5125CC4B4B2
:106800008D030279E2024C09122EAB124D81BF00BA
:106810000DB4C8005008F57090BF6DE0600C306496
:1068200006124AC202644A024C0F20480330600E2E
:106830001251AF4009E570B4BE00500280E0124929
:10684000016008E55E7004C26080D3E570125905EE
:10685000406EE570124C34E9F404F56FE57012599E
:10686000D55004C26080B785707ED260124AB730BE
:10687000640F12511A7431125CCFE55E6029026810
:1068800091E55E700612511A0268A7124E2C125141
:106890001AE55E6012E57E12591E124901600DE58F
:1068A0007E1259180268B1E57E12596AE57E1259C6
:1068B00064D25F306406122E8302656B755D002220
:1068C0007429122F59E5701251E9124E5E75710349
:1068D000755D04024AC61249375010124AB7157145
:1068E000122EABE57160012202680BB40B09E57151
:1068F000640370230266C2B4120FE571640370175B
:10690000124AB775710002685220640B124AB7E54B
:106910005C755D00025FED02681EE55CB4110F124C
:106920005CC4B48D030279E2024C09024C0FE55BB2
:10693000906936020B6C0269420269550269630272
:10694000698812493750E4124AB7749B122F59755F
:106950005B01022EAB12493750D1124AB7755B0268
:10696000022EAB12493750C3124AB7122EAB124D4A
:1069700081BF00B7B4C80050B2F57090BF6DE07031
:10698000AA12508B755B0322E55CB4129E124AB7C3
:1069900085707E124973124E2C124C36E9F404F5C0
:1069A0006FE57E1259D5E57E125964E57E12596A6B
:1069B000024C14E55CB40B1D124973C259124AB75C
:1069C000741C122F59C25612788F755D0E755B00BC
:1069D00074A1025CCF500C122EAB125CCD755D061B
:1069E000024AB7B415030269ECB4142B90BF6DE0F2
:1069F000B40303026AFA741A122F597430122F4A20
:106A0000122F4A122F52757103124E4E757E007569
:106A10005D08D25F024AB7B40C030270E1B4131AE6
:106A2000124AB7E55E70061249A4024C171249FFDC
:106A30007FF07490122F68024C17B4110C125CC4D2
:106A4000B48D030279E2024C09B43505C2590265DE
:106A5000E7026AFA1249374003026ACC124AB712B7
:106A60002EAB755D07025CCD124937504D122EAB2F
:106A7000124969124D81BF00D8B4C80050D3126BBF
:106A80000E5003026AFA124AB7C24830591690C033
:106A90005EE0655E7005055E105913E57EB4BE00CC
:106AA0004002D248D26012511AD25F024C17124AE9
:106AB000C2127501125CCD024C17B40D0C90C0834C
:106AC000123143124DB0026AD7026AEBB40D1C12A8
:106AD0005CE0B40A027400126B0E401E126A891246
:106AE0005CC4B41B02800302614222B4110C125C2C
:106AF000C4B48D030279E2024C09124AC2C2593071
:106B00007109124F1C125CCD024C17024C14F57E19
:106B100090BF6DE05403B40303026B74B4020040F1
:106B20000AE57EB40A004003026B74E55E122E7221
:106B3000B40C2590C05EE55E14F0D259E57E124D8E
:106B4000C0403190C05EE025F0D271B421005024E5
:106B5000C271124DF4026B5FC259E57E125A0D12DA
:106B60004E1EE55E6012124C36E9256F600A12492E
:106B70006C125D5EC260D322C256C32212493750E6
:106B80003AE5717003026C35124AB71571E5716010
:106B90001AB40211741A122F597D007E00AF5C12D4
:106BA0004D87026BB6124DAA026BB6124D81B4C866
:106BB000004003024C0FF57E022EABB41532124A90
:106BC000B78002057E90BF6DE0B40207E57EB40A8F
:106BD000005007E57EB4C8004007205F5B7400F5F5
:106BE0007E12590550DDE57E126B0E40D6026C1701
:106BF000B4142F124AB78009157EE57E7003205F1A
:106C000037E57EB4FF03757EC7E57E12590550E86F
:106C1000E57E126B0E40E1126A89C25F755D090262
:106C200057D1B41110D25FC260125CC4B48D03029C
:106C300079E2024C09024AC2127501125CCD024C83
:106C400017E55CB41509124AB7126C64026BC3B441
:106C50001408124AB7126C64809ED25F124C17E57A
:106C60005C025FB7755D08AE5E90C05EE0FCCEC3AF
:106C70009ECE8C5E7400122E2EDEF98C5E740C0299
:106C80002E2EE55CB40B2F124AB77497122F619029
:106C9000BEB7E0B40A004004E4122F82122EA5C24F
:106CA00056C260C248125D5E12788F755D1B755BBF
:106CB0000074A1025CCFB4110C125CC4B48D030249
:106CC00079E20263FD125CC4B41D0312994EE55CC7
:106CD000B40D03026142B40E0302638D024AC2E5A1
:106CE0005CB4110C125CC4B48D030279E20263FD42
:106CF000B40E0302638DE55B906CFE020B6C026DBB
:106D000007026D64026E09125CC4B41C3CE55CB4FD
:106D10000B2A124AB790BF23E0A2E09260A2E19250
:106D20004890BF5DE0F57E74CD125A0D124E1E7470
:106D30001D122F59C256755D0A025CCD74A1122F27
:106D400059125CC9C25E024AC2E55CB415028003F6
:106D5000B414F3124AB7C260C248755B0190BEB862
:106D6000E0026D85E55CB4150E124AB7E57004B417
:106D700005004011E4800EB4146C124AB7E570149B
:106D8000B4FF027404F57024C8125A0D12519740D2
:106D900005124A5080031249FF90BEB8E0C39570B7
:106DA0005002240504601A906DBE23232582F582CB
:106DB000E43583F58379007A03124EA4743A022FE6
:106DC00052223173743A326E643A3372643A3474D4
:106DD000683A3574683A3674683A3774683A387481
:106DE000683A3974683AB4130B124AB7755B027487
:106DF000A2022F59B40D06124C14026142B41203C0
:106E0000026423B41A1F026563E55CB41317124AC7
:106E1000B7755B01E55E600A1249FF74907FF0026E
:106E20002F68026D96024AC2E55CB4110C125CC474
:106E3000B48D030279E20263FDB40E0302638DE5B3
:106E40005B906E47020B6C026E50026EA8026F14CC
:106E5000125CC4B4972DE55CB40B1B124AB71258F0
:106E60004312788F749F122F59C256755D1C755B43
:106E70000074A1025CCF74A1122F59125CC9C25ECA
:106E8000024AC2E55CB415028003B414F3124AB797
:106E900090BEB7E0F570600AC260C248755B01023F
:106EA0006ED2124AC20263FDE55CB41513124AB7F2
:106EB000057090BEB7E0B570005017757001801274
:106EC000B4142E124AB71570E570700690BEB7E084
:106ED000F570E57024CD125A0D1251974005124AF3
:106EE0005080031249FF90BEB7E0C3957004026D55
:106EF000A5B4130B124AB7755B0274A2022F59B4E2
:106F00000D06124C14026142B41203026423B41A37
:106F100018026563E55CB41310124AB7755B011281
:106F200049FF74907FF0022F68024AC2E55CB411F9
:106F300015125CC4B48D030279E2E55BB4040280EF
:106F40000BD25F0263FDB40E0302638DE55B906FAD
:106F500054020B6C026F63026FA3026FDA02703B84
:106F600002709A125CC4B49F15E55CB40B0302690D
:106F7000BD74A1122F59125CC9C25E024AC2E55CFF
:106F8000B413028003B4140C124AB7757000757202
:106F90004102700EB415E4124AB775701D75727A0D
:106FA00002706DE55CB413028003B41406124AB794
:106FB000026FFFB41506124AB7027060B40D0BD20F
:106FC0005F124C1712511A026142B4120A755B0427
:106FD000124AB712504822024AC20572E572B47BC7
:106FE0000050057570008026305F0C1249691275DB
:106FF00001125CCD024C17757000757241800F054F
:1070000070E570B41E004006755B020257D6E5704D
:1070100012584A50EAE57012589DE572B45B004080
:1070200002943BF8E06870D7E5701257F5125822C9
:10703000C25F755B011257DB025CCD1572E572B45D
:107040004100400575701D8024305F0C12496912A3
:107050007501125CCD024C1775701D75727A800D2A
:107060001570E570B4FF06755B030257D6E5701224
:10707000584A50ECE57012589DE572B45B0040022E
:10708000943BF8E06870D9E5701257F5125822C2A7
:107090005F755B011257DB025CCDE55CB412321206
:1070A0004AB7125843125D5EE57012585CE57012E3
:1070B000585690BE747F04E07011125A4FDFF812D8
:1070C000788F127501125CCD024C17755B01026F4F
:1070D000FFB41105124AB780B3024AC2E55CB40C92
:1070E0000C124C4612788F755D10024AB7B4110924
:1070F000125CC4B48D090279E2B40E0602638D02FB
:107100004C09024AC2E55CB40C09128577755D0B27
:10711000024AB7B41109125CC4B48D090279E2B411
:107120000EE002638D024C09E55CB40CC0124AB754
:10713000741FA2129400122F59755D0C90C090021A
:107140005636E55CB40CA67420122F59125609125B
:10715000494312561B755D0D024AB7E55CB40C8DB0
:10716000124E9A90BF3A12561B755D0F024AB71223
:1071700049691251974006124A500271801249FF24
:107180007F327422022F68C25EE55B5407907193D0
:10719000020B6C0271AB0273E00274310274810263
:1071A00074900271AB0271AB0271ABE55CB40D007F
:1071B000400302726C305F0712716FC25F801F1252
:1071C0005CE0B40D004007124A9760128004655CD1
:1071D00060120571E571B4080040037571077570A0
:1071E000000271E9057053700312491775F004E548
:1071F0005CA4257090720830260390723893FF12B9
:107200004911EF122F52124917024AB7515A26312B
:107210004142433244454633474849344A4B4C3552
:107220004D4E4F365052533754555638575859399A
:107230002B2829302A2E3F27232F2D3D717A2631E6
:107240006162633264656633676869346A6B6C35A2
:107250006D6E6F36707273377475763877787939EA
:107260002B2829302A2E3F27232F2D3DB41A2012F8
:107270004AB7124E1E124C17757000D25FE55E7051
:107280000B1249016003024F290249A402645CB455
:10729000113C125CC4B48D0612656B0279E2124A8D
:1072A000B7026563124A977012E571601B124917A5
:1072B000122F501571E5717002C226124917745FC2
:1072C000122F527F001249111249170257D6B413D8
:1072D000030272D7B41B23124AB7757000D25FC283
:1072E000261249016008F571755D120274CA757243
:1072F00041757101755D13027584B4152F124AB77B
:10730000305F0512716FC25FE571B4070040030280
:107310004AC2124A97700B7F201249111249171264
:107320002F500571124917745F022F52B41429129D
:107330004AB7305F1012716FC25F124917745F1243
:107340002F52024AC2E5717003124AC20272A4E5CA
:107350007160021571024917B41266205F1F12494D
:107360000160DFD25FC226124AB7124E1EE55E7080
:1073700006755B01024F29755B020250D47C001236
:1073800073B1401C124AB7125843125D5E12788FD7
:10739000755D1E755B0074A0122F597432025CCFAC
:1073A000124AC212788F742A122F59125CCD024CE5
:1073B00017BC1E00B34009EC12584A50030C80F170
:1073C00022B41619124A97600BE571B407005008F1
:1073D00005718004E5716005B226024AB7024AC20F
:1073E000E55CB40D00500A1260DC755D11755B013F
:1073F00022B4120EE55E6036126423755D11755B72
:107400000222B40E06E55E70DE8023B41A03027217
:107410006FB4111AE55E6013B4020040051263DA1E
:1074200080C8125D5E1273EA024F29026563024A48
:10743000C2124937500A1266BD755D11755B032291
:10744000B4120BFF125CC4B42931EF0268F7B40B1D
:107450000D1266BD125CC470A27431025CCFB41A06
:107460000302726FB41103026563B40C0E124AB7C3
:107470007498122F5975700002678B124AC2026508
:107480006612493750D81267D4755D11755B0422B6
:1074900012493750C91267F4125CC46012B4280351
:1074A0000273FBB42A030273FB755D11755B022244
:1074B000E55CB41351124AB7205F0F0570E570B454
:1074C000C8004006205F37757000AE71E570125835
:1074D000FF50E8E570129DC97872E06670DD081211
:1074E0005A4FDEF6AD71E570126B0E8D7140CCD245
:1074F0006012511AD264C25F755D120257D1757065
:1075000000741B022F59B40D0050061265630271FE
:1075100087B40D09124C1712511A026142B4110FAF
:10752000125CC4B48D0612656B0279E2026563B425
:107530001603024AC2B41503024AC2B41403024A33
:10754000C2B41203024AC2B41A10124AB7124E1E33
:10755000757000D25FC264024C14755D11027187B0
:10756000E55CB4130302756BB41B9B124AB7205F32
:107570006B0570E57075F01484E5F07007755D13A8
:107580000257D622E5701258FF50E6E570129DC9E9
:10759000E572B45B004002943BF8E06870D3AD71D3
:1075A000E570126B0E8D7140C8D26012511AD26410
:1075B000C25F755D140257D1E570B4C80040C505BF
:1075C00072E572B47B00500575700080B7305F0CB7
:1075D000124969755D141257D102750175700075F5
:1075E0007101757241809DE55B9075EF020B6C0235
:1075F00075F5027676E55CB41134125CC4B48D0680
:107600001276060279E2205F1C124AB7E55EB402E8
:1076100000400812497ED25B0257D1D25F125D5EF4
:107620007432022F59124AB7124C170249A4125C45
:10763000C4B4A00B127620125CC9C25E024AC2E535
:107640005CB41219205F2C124AB712788F1258437B
:10765000D264C2267431122F59755B0122B40B001B
:107660005011305F05C25F122F58E55E640B600356
:107670000260DC024AC2E55CB40D0040030276D72A
:10768000305F071277D5C25F801F125CE0B40D0037
:1076900040071277CE60128004655C60120571E5C8
:1076A00071B41000400375710F7570000276B40557
:1076B0007053700312491775F004E55CA4257090AF
:1076C000720830260390723893FF1277C8EF122F9A
:1076D00052124917024AB7B41121125CC4B48D0684
:1076E0001276E60279E2205F03027647124AB71269
:1076F000788F125843124C170249A4B4152F124A1E
:10770000B7305F051277D5C25FE571B40F00400353
:10771000024AC21277CE700B7F201277C812491727
:10772000122F500571124917745F022F52B414477B
:10773000124AB7305F101277D5C25F124917745FD3
:10774000122F52024AC2E5717003124AC21277CE5A
:107750007012E571601B124917122F501571E571F7
:107760007002C226124917745F122F527F001277DF
:10777000C81249170257D6B41232205FC678DEB657
:10778000000280BF757000C226AC701273B140B3A6
:107790008C70124AB7E57012585CE5701258507C34
:1077A000001273B140030273840273A3B4169412DF
:1077B00077CE600BE571B40F00500805718004E5C9
:1077C000716080B226024AB71277CEEFF622E571D9
:1077D00078DE024AA27401122F5974CD025CBF12E6
:1077E0005CC4B43E03027894B41303027894124844
:1077F000ED02785D7873E66416702E08E6640A7010
:107800002808E6640B702208790290AE2BB60B00B4
:107810005017E6C408B60B00500F46FFE06F700922
:1078200012309708D9E702788A204C3090C082E065
:1078300064097028A3E064017022A3E06401701C55
:10784000A3E0640D7016C256C260757000125D5ED2
:10785000755F91756010755E030262BA22797912C4
:1078600078AB6011E55CB435030265E7B40E853092
:107870004F8202637D1257BA12788F125CC4B42E05
:1078800006124C170257AE024C14D2671250E8D2BF
:107890005F02496912493750030294B4B4120620BA
:1078A0005F03128429124C280250ED90BF5FE0FF65
:1078B000EF122E8A67700319DFF622E55B601678F7
:1078C0005CB61111D25FC25AC25C124C09125CB88C
:1078D00060E8028C3DB4080040047400F55B9078C9
:1078E000E4020B6C0278FC02795002795E02797E28
:1078F0000279940279A90279C20279DD907946E58C
:107900007193B55C3BE570B40123125CB87003124F
:1079100060DCD25AC25C7485122F59748C125CCF11
:10792000755B0112788F125D5E755D1522125CB871
:1079300070031260DC15700571755D15755B0022B2
:10794000124C17025FDC0B08030708060603030C42
:10795000E55CB414030279E2B4151D0279C7E55C55
:10796000B4140DC25C124AB7124EC6755B0380B9DF
:10797000B41505C25C0279C71279E5024AC2E55C1A
:10798000B4140B124AB7124EE5755B04809BB41514
:10799000EA0279E2E55CB4140B124AB71286277545
:1079A0005B058085B415D480BAE55CB4140F124A27
:1079B000B71250B6129498755B06027929B415BBBC
:1079C00080C1E55CB41411124AB7127E9FC25E12E8
:1079D0005CC9755B07027929B415A080BCE55CB46D
:1079E0001412124AB7124EC1D25C755B0278C87687
:1079F00015027929B4158480B578CEE67003027A31
:107A00007DE55CB41611E570640670F212654BC238
:107A100065757005027A79B40D0FE5706405705DC7
:107A2000124AB7757004027A79B40E0FE5706404D7
:107A3000704B12637D757003027A79B4130FE57091
:107A400064037039126465757002027A79B4120F9A
:107A5000E57064027027126423757001027A79B4AC
:107A6000111BE570640170151263DA437A8075703A
:107A7000007486122F59024C17755D162278CE7647
:107A800000755D00125CB86003755D18025FDCE58F
:107A90005A04C39402907A9B020B6C027BC6027E4E
:107AA000F3027C8A027CBA027CEB027D1B027D54CD
:107AB000E55AB40C0040047400F55A907AC1020BE8
:107AC0006C027AF4027BC1027C2C027C7E027CAECA
:107AD000027CDF027D0F027D48027DA3027DFB0256
:107AE0007E41027EE0755A08027DA3755D1502781D
:107AF000FC0278FC78CEE670028082E55CB4350347
:107B00000265E7B40D0050F1E570B40A08E55CB415
:107B10000BD3027BA4B40926E55CB40603027BA464
:107B2000B4080280C690BEDAE070BA125CB8700881
:107B3000E55CB401B60286C3124C17025FDC907B91
:107B4000B7E57193B55CB2E570B40158125CB870DA
:107B5000031260DCD261C27C7490122F599000181D
:107B6000740093122ED5900019740093122ED51222
:107B70004E4E90BEC27903122DFCE0122ED5122E6D
:107B800001A3D9F3E0122EB9755D19755A09755B19
:107B9000007482206105755A0A7499D221D24EC2AE
:107BA0007C025CCF125CB870031260DC157005714A
:107BB000755D19755A00220B0602070209080504B3
:107BC0000CE55CB4141B124AB77405122F59745794
:107BD000125CCF79011231EC755A02755B000257C5
:107BE000D1B41506124AB7027D80B41121125CC4CB
:107BF000B404D3125D5E124C09D25F90BF2CE0F941
:107C00001231ECC221E55DB418030250ED22125C82
:107C1000C4B45712E55CB40B0D124AB7125A5B128A
:107C20004F12740580AA127D6D024AC2E55CB4143D
:107C30001B124AB774B0122F597431125CCF7901FC
:107C40001231EC755A0B755B000257D1B415061250
:107C50004AB7027D6DB41108125CC4B405D3809399
:107C6000125CC4B45712E55CB40B0D124AB712058E
:107C7000C4124F1774B080C3127BC6024AC2E55BC0
:107C8000600302805BE55CB41413124AB7740712F8
:107C90002F5979021231EC755A04027D2BB415026A
:107CA000808FB41103027BF3127EF3024AC2E55BBC
:107CB000600302805BE55CB41413124AB7740812C7
:107CC0002F5979031231EC755A05027D2BB4150337
:107CD000027EF3B41103027BF3127C8A024AC2E5EE
:107CE0005B600302805BE55CB41413124AB774094D
:107CF000122F5979041231EC755A06027D2BB415F6
:107D0000028087B41103027BF3127CBA024AC2E5F7
:107D10005B600302805BE55CB4141B124AB7740A13
:107D2000122F5979051231EC755A07755B007421D1
:107D3000125CCF0257D1B41503027CBAB41103020E
:107D40007BF3127CEB024AC2E55B600302805BE5D9
:107D50005CB4143D124AB779011231EC3061211242
:107D60004E737457125CCF755A090257D1740412BE
:107D70002F597457125CCF755A01755B000257D1A9
:107D8000127E9F7457125CCF755A0A755B000257BA
:107D9000D1B41503027CEBB41103027BF3127D1BFB
:107DA000024AC278CEE67003027A7DE55CB40D002B
:107DB00050F690BEDAE571C3132582F58274003562
:107DC00083F583E0F5F0E57113E5F04001C4540F4D
:107DD000B55CD5E570B40110125CB870031260DCBC
:107DE000C261027B56027A7D125CB870031260DCBD
:107DF00015700571755D19755A0822125CC464907E
:107E00006039E55CB41406124AB7027D80B41503EC
:107E1000027D1BB41109125CC4B482EE027BF31222
:107E20005CC4B45716E55CB40B11124AB7124E3A53
:107E30007483122F59755B00027B96127D57024A9C
:107E4000C2125CC464906051E55CB4141B124AB762
:107E50007404122F597457125CCF79011231EC75EA
:107E60005A01755B000257D1B41509206103027DE8
:107E70001B027D54B4110A125CC4B499D0027BF386
:107E800022125CC4B45712E55CB40B0D124AB7124F
:107E90007ED3125028740480BE127D80024AC274C0
:107EA00099122F5990BEDF122DFCE06025122EC3CF
:107EB0007C03122E01125A4F122DFCE0122ED5DC3B
:107EC0000A122E01125A4FE0022EB9742D122F4AB7
:107ED00080E02290BEDF7A050207237403022F5947
:107EE000E55B907EE8020B6C027EEE027F20E55C93
:107EF000B4141B124AB77406122F597421125CCFA6
:107F000079011231EC755A03755B000257D1B41533
:107F100003027BC6B41103027BF3127C31024AC216
:107F2000E55CB40D004003027F80305F07127EDB0A
:107F3000C25F801F125CE0B40D004007124A9760D8
:107F4000128004655C60110571E571B4080040039E
:107F500075710775700080050570537003128053AA
:107F600075F004E55CA425709072083026039072C9
:107F70003893FF124911EF122F52128053024AB761
:107F8000B4111A124AB7305F07C264C226027EF3E8
:107F9000126566755D19755A0B755B0122B4152F54
:107FA000124AB7305F05127EDBC25FE571B407008D
:107FB0004003024AC2124A97700B7F2012491112E5
:107FC0008053122F500571128053745F022F52B4E8
:107FD0001447124AB7305F10127EDBC25F12805323
:107FE000745F122F52024AC2E5717003124AC21224
:107FF0004A977012E571601B128053122F50157151
:10800000E5717002C226128053745F122F527F00F6
:108010001249111280530257D6B412181249016046
:10802000C490BEAF78727C08124B8AD25FC264C221
:1080300026027EF3B416AE124A97600BE571B407C0
:1080400000500805718004E5716005B226024AB748
:10805000024AC2E5712408F9024E60E55BB40A00E9
:1080600040047401F55B90806C020B6C027AB002E4
:10807000808A0281B302825A0282D002833C028348
:10808000B00284380284A902850BE55CB4140612A0
:108090004AB7028577B4150E124AB7E55AB40303FE
:1080A0000286620285B7B41126305F030281867FA3
:1080B0000978787979124D707700155EE55E700267
:1080C000D25F124AB7747F122F52D25B0257D1B4DB
:1080D000126F205F66E55EB40A0050030281837868
:1080E00070790412818990C0F6ED543FF0A3EE54EC
:1080F000F0FEE0540F4EF07873790212818990C03F
:10810000F7ED540FFDE054F04DF0A3EE54FCFEE506
:108110007604030354034EF0A3787779041281891F
:10812000ED543FFDE57604030354C04DF0A3EE5437
:10813000F0F012057312819112057A124AB7028586
:108140006EB40B00503D305F08C25F755E00125088
:10815000CFE55EB40A00502B122EAB7F09787179FF
:1081600070123023E55C785BB6010714F7055E02F8
:108170004AB7B6060280F5B6090280F0B40AED747B
:108180000080E9024AC2027A8F1281A2E9FF024D01
:10819000771281AC7C0590C0F6122DFC1231A8023A
:1081A0003210123152124D87FEEFFD22E55AC39470
:1081B00002F922E55CB41406124AB702858AB415A6
:1081C00006124AB702856EB411030280A9B41247A1
:1081D000205F3E128234E57679E87803124D64E53B
:1081E0007579107827124D6412824290C0F4ED54D4
:1081F0007FF0A3EEF090C0FB7401F0A3EEA2E0B319
:10820000744D3400F01205731282491282BF1205B8
:108210007A124AB7028577B40B005015305F08C256
:108220005F755E001250F7E55EB4050050030281F1
:1082300058024AC278771281A2EDFAEEFB7D007EE9
:108240000022EE2BFEED3AFD221281AC7C0290C0A2
:10825000F4122DFC12317C023210E55CB4140612CB
:108260004AB702859BB41506124AB7028577B41146
:10827000030280A9B4122B205F22128234E57679A2
:10828000E87803124D6412824290C0FBED5407F06F
:10829000A3EEF01205731282BF12057A124AB702DA
:1082A000858AB40B005015305F08C25F755E0012FE
:1082B00050ACE55EB404005003028158024AC21279
:1082C00081AC7C0290C0FB122DFC1231B90232103D
:1082D000E55CB41406124AB70285B7B41506124A13
:1082E000B702858AB411030280A9B41221205F1855
:1082F000A979E57875F00AA429540F90C0FDF01211
:10830000057312832B12057A124AB702859BB40BB0
:10831000005015305F08C25F755E001250B1E55E17
:10832000B402005003028158024AC21281AC7C019F
:1083300090C0FD122DFC1231CA023210E55CB4145B
:108340000E124AB7E55AB403030285D302856EB410
:108350001506124AB702859BB411030280A9B41214
:1083600021205F18A979E57875F00AA429540F90A7
:10837000C0FEF012057312839F12057A124AB702EB
:1083800085B7B40B005015305F08C25F755E0012F0
:1083900050BBE55EB402005003028158024AC2128B
:1083A00081AC7C0190C0FE122DFC1231DB02321038
:1083B000E55CB41406124AB70285EEB41506124AFB
:1083C000B70285B7B411030280A9B4122AE55EB4DE
:1083D000043F205F1C12841412057390AE2BE571CC
:1083E000122F82123097E572122F82125C751205DD
:1083F0007A124AB70285D3B40B005015305F08C219
:108400005F755E001250B6E55EB404005003028151
:1084100058024AC27876128433FD08128433FE1261
:1084200049697570048D718E72787090BF5F7C079A
:10843000024B8AE6C408D622E55CB41406124AB799
:10844000028627B41506124AB70285D3B411030277
:1084500080A9B41224205F1BE55EB4043A12849A0A
:10846000540FF912057390ADEBE9122F82125C756F
:1084700012057A124AB70285EEB40A03028482B466
:108480000115305F08C25F755E001250C0E55EB432
:1084900004005003028158024AC2A97678777F030C
:1084A000E613E933F908DFF822E55CB41406124A52
:1084B000B7028662B41506124AB70285EEB41103FC
:1084C0000280A9B41224205F1BE55EB4043A128432
:1084D0009A540FF9120573E990AEAB122F82125C19
:1084E0007512057A124AB7028627B40A030284F38A
:1084F000B40115305F08C25F755E001250C5E55EBD
:10850000B404005003028158024AC2E55CB4140668
:10851000124AB702856EB41506124AB7028627B40E
:1085200011030280A9B41229205F2012057390AFB5
:108530002B12309778747C03E6C408D6122F82126F
:10854000309708DCF3125C7512057A124AB702867E
:1085500062B40B005015305F08C25F755E001250A8
:10856000CAE55EB406005003028158024AC2124CAA
:1085700046755B0102788F7410122F59124CFB7EE6
:1085800004128686755B0202788F1250AC124D423F
:108590007E03128686755B0302788F1250B190C0FD
:1085A000FDE0540F75F00A84ADF0122EC9ED122EC5
:1085B000AD755B0402788F1250BB90C0FEE0540F83
:1085C00075F00A84ADF0122EC9ED122EAD755B0563
:1085D00002788F1250B690AE2BE0FD123097E0FE7D
:1085E000ED122ECFEE122EB3755B0602788F12506D
:1085F000C012788F90ADEBE0540F30E30375730138
:1086000030E20375720130E10375710130E00375EA
:1086100070017E037973E7122EC919DEF9E7122E75
:10862000AD755B0702788F1250C512788F90AEAB94
:10863000E030E30375700130E20375710190AEAB79
:10864000E030E10375720130E0037573017E037958
:1086500070E7122EC909DEF9E7122EAD755B08022C
:10866000788F1250CA90AF2B1230977902122DFCDE
:10867000E0122ECF122E01123097D9F1E0122EB354
:10868000755B0902788F7970E7122EC909DEF9E768
:10869000022EADE55B90869B020B6C0286A40286DF
:1086A000E102875E9086D7E57193B55C24E570B4EE
:1086B00001111260DC7480122F59755D17755B0112
:1086C00002788F1260DC15700571755D17755B009F
:1086D00022755D00025FDC0B01020304050607083A
:1086E0000CE55CB41121124AB7205FC975F000781F
:1086F0005E7970E6122E60155EE55E60030280C54D
:10870000E55BB4012180AEB41226305F031287A965
:10871000E55EB40A0040447870795F7C05E6F708AE
:1087200009DCFA124AB7D25F755B027481022F59D5
:10873000B40B005026305F0AC25F755E00748B1266
:108740002F59E55EB40A005012122EAB7970785E94
:10875000E6855CF0122E6006024AB7024AC2E55C6A
:10876000B41108124AB7205FBD8081B41233305F64
:10877000031287A9E55EB40A0040287870795F7C0F
:1087800005E766701E0908DCF8787090BEDA7C0593
:10879000124B8A12788F122E83124AB7C261027B63
:1087A00056808D124AC20286B5785E76009086D7D2
:1087B0007970E693F5F0E6122E6006B60A0040F0F6
:1087C00022124930700EE55AB401033052069087E8
:1087D000DC020B6CE55A9087EB020B6C02880902F5
:1087E00088190288C80288FA02894E0289700289B3
:1087F00076028A09028A54028AD0028BD2028C5FE6
:10880000028CC402908F029618124AB7D25FD252DD
:10881000755A011250D90257D1E55CB417004021B6
:10882000B41A061259B0026563B421091259B01284
:1088300065A9028849B422171259B01265AE0288A0
:1088400049B40D00500A1260DC755D1A755A042295
:10885000B41103028858E55CC3940D908861020B43
:108860006C02887F02637D02884F02884F02888CE9
:108870000288C20288BC0288920288A502889212ED
:1088800059B0124B005070C252024C14205F5F026C
:1088900063DA1259B0C252124AB7D2631250DE756F
:1088A0005A020257D1124AB71259B0C252D2517568
:1088B0005A03125CE578C8760A0257D11259B00201
:1088C00064651259B0026423E55CB416030288D3D0
:1088D000B41404C26380CEB41505C263028905B422
:1088E000110F125CC4B48D061289370279E2028935
:1088F00031B40E0302638D024AC2E55CB416030272
:108900008905B41412124AB7C251D25FD252755AB5
:10891000041250D90257D1B41508124AB7C25102F5
:108920008892B41120125CC4B48D06128937027982
:10893000E2128937024C091259B0C252C263C251C5
:10894000D25F024E2CB40E0302638D024AC2E55C74
:10895000B40D191259B078C0E670147411242AF6B7
:10896000D249D25F124AB7C252024C14028819226D
:1089700012657F0257D1E55CB417004016B4350F7D
:10898000C267C265D25F124E2C124C140265E70218
:108990004AC222B40B00500B125D5EE55C122E2E13
:1089A0000261F3940B9089AB020B6C024AE3024A1A
:1089B000E30289F802637D0289920289920289EDBD
:1089C000024AC2024AC20289CF0289E00289CF125A
:1089D0004930700302654BC2651288A5755A0222A0
:1089E000124930700302654BC265028D171249307F
:1089F000705412893E024C09126142125CC4B43BAD
:108A000007E55E600302511A22E55CB41603028A90
:108A100014B41418C251124AB712788F7474122FFA
:108A2000597475125CCF755A030257D1B41508C238
:108A300051124AB7028970B41117125CC4B48D0682
:108A4000128A4C0279E2128A4C024C09C2650289F0
:108A50003E024AC2E55CB41603028A5FB4141A12DD
:108A60004AB712788F90BEB9E05403F570128B3478
:108A7000755A04755B000257D1B415030289CFB44F
:108A8000110E125CC4B48D06128A4C0279E280B6D3
:108A9000B4132A124AB7E570B40A05124FA480171E
:108AA000B40D05124F7B800FB40E05124F56800790
:108AB000908AC093122F59057053700F22024AC238
:108AC0007D7E7B7C89797AAAAB78B376ACB2B17FB4
:108AD000E55CB41603028ADBB41414124AB71278A8
:108AE0008F743D122F59755A05755B000257D1B42A
:108AF0001503028A14B4110F125CC4B48D06128AD5
:108B00004C0279E2028A46908B11E55B540125E024
:108B1000738002805DE55CB41327124AB7E57004E8
:108B20005403F57078DBE620E20AE570B4030040F8
:108B300003757000E570B40203024F3B24A3022FBB
:108B400059B4122B124AB7E5705403F570700D90AA
:108B5000BEB9122F82C2461234238082B4030302AC
:108B60008BA090BEBAE0F571128BC4755B01220236
:108B70004AC2E55CB41243124AB7E57190BEBA121C
:108B80002F82E570B4011190BF31E030E705741811
:108B9000122F82123423801590BEB77400122F82D8
:108BA0007D467E5090C09312315B12340AE570907E
:108BB000BEB9122F82D246028ADEB405005010F5EB
:108BC00071124AB712500AE571122EA5024E5E02CA
:108BD0004AC2908BDCE55B540125E0738002805132
:108BE000E55CB41603028BEBB4141B124AB712787F
:108BF0008F90BF5BE0A2E792E05401F570128CA267
:108C0000755A060257D1B41503028A5FB4110F12C8
:108C10005CC4B48D06128A4C0279E2028A46B40A18
:108C20000D124AB712788F1250E8755B0122024A82
:108C3000C21248DD70F779791278AB701C30460D9E
:108C400090BEB9E0B40106E4122F82C2461250ED84
:108C500012788F1257C3024C17128A46024BFBE55B
:108C60005CB41603028C6AB41414124AB712788FDB
:108C70007444122F59755A07755B000257D1B41509
:108C800003028ADBB4110F125CC4B48D06128A4C45
:108C90000279E2028A46B4130E124AB7E570B2E0D6
:108CA000F5702448022F59B41217E570A2E092E73C
:108CB0005480F57090BF5BE0547F4570122F828026
:108CC000A9024AC2E55C785BB41115125CC4B48D8C
:108CD00006128CD70279E2B60003028A46028D178B
:108CE000E6540F908CE9020B6C028D0D028D390257
:108CF0008D94028E1B028E6D028ED2028F2B028FFC
:108D00007B028F93028FAC028FEA029044E55CB441
:108D100016028003B41413124AB7745C122F5975EB
:108D20005A08755B00D25F0257D1B41503028BEB72
:108D3000B4130302904E024AC2E55CB416028003EB
:108D4000B41416124AB712788F7440122F5974CA8D
:108D5000125CCF755B020257D1B41503028FB6B413
:108D60001315124AB70570E570B40300400474008F
:108D7000F5702452022F59B412171257EE7008E5FD
:108D80007013B3926AD24790BF74E570122F82803D
:108D9000B2024AC2125CC4B4CA3FE55CB416061201
:108DA000495E028DE3B41403028DAEB41509124975
:108DB000621257D1029CF1B4110612495E0263DAC5
:108DC000B4120D90BF36E0045403122F82024962A0
:108DD00012495E124AC2028D49E55CB41602800354
:108DE000B41417124AB712788F90BF34E05403F5C9
:108DF00070128E50755B030257D1B4150302904E6A
:108E0000B4110F125CC4B48D06128A4C0279E202CE
:108E10008A46B412BB124962025115E55CB41602CF
:108E20008003B41417124AB712788F90BF73E054BE
:108E300003F570128EBD755B040257D1B4150302A1
:108E40008D43B41310124AB70570E5705403F570E2
:108E5000244E022F59B41212E570700490C0F1F044
:108E600090BF34E570122F8280BB024AC2E55CB429
:108E700016028003B4141B124AB712788F90BF37C2
:108E8000E0A2E792E05401F570128F09755B0502CC
:108E900057D1B41503028DE3B4110F125CC4B48D25
:108EA00006128A4C0279E2028A46B41315124AB7B6
:108EB0000570E570B4030040047400F570244102AD
:108EC0002F59B4120A90BF73E570122F8280A80246
:108ED0004AC2E55CB416028003B4141B124AB712EE
:108EE000788F90BF5EE0A2E492E05401F570128F9B
:108EF00050755B060257D1B41503028E25B4130ECC
:108F0000124AB7E570B2E0F570244C022F59B41242
:108F100017E570A2E092E75480F57090BF37E054F7
:108F20007F4570122F8280B4024AC2E55CB41602FB
:108F30008003B41409124AB71265930257D1B415CD
:108F400003028E77B4130E124AB7E570B2E0F570E3
:108F5000244A022F59B41220124AB7E570600C124D
:108F6000788F1250E8755B070257D190BF5EE054CE
:108F7000EF4570122F8280C0024AC21248DD701283
:108F800079791278AB700575701080DF128A46020D
:108F90004BFB22E55CB4140B1265900257D174951B
:108FA000022F59B41503028EDC024AC2E55CB416E6
:108FB000028003B41417124AB712788F90BF5BE097
:108FC0005401F570129077755B0B0257D1B41503FD
:108FD000028EDCB4130C124AB7755B0A757000027E
:108FE00090037472122F59024AC2E55CB4160280D3
:108FF000C5B4140280C0B4150280D2B41330124A32
:10900000B70570E570B4C800501912590540F274E4
:1090100087122F59C25F124E42E5701251E978C78C
:109020007605227570FF305FD8742A022F59B4126A
:1090300008205F0DE570026811C25F124C17025FD5
:10904000ED024AC2E55CB416028003B41417124A5A
:10905000B712788F90BF74E05403F570128D72755B
:109060005B010257D1B41503028F35B4130E124AB7
:10907000B7E570B2E0F5702458022F59B4120D9084
:10908000BF5BE054FE4570122F8280C2024AC2E5E7
:109090005C785BB41124125CC4B48D061290A202F9
:1090A00079E2B600028010205F42B60500403DB66E
:1090B0000A0040060290EC028A46E55B540F90904D
:1090C000C4020B6C0290E202910C02913202919D5B
:1090D00002922102929C02933F0294290294D502AB
:1090E000959BE55CB416028003B41406124E2C0264
:1090F000654BB41503028C6AB4130E124AB7743070
:10910000122F59755B0102788F024AC21248BF4084
:1091100020124A6830D506128A46024AC212788F57
:1091200090BF2CE05407F57012916C755B020257EA
:10913000D122E55CB4160302913DB41416124AB76D
:1091400012788F7455122F597456125CCF755B03C9
:109150000257D1B4150302934AB41315124AB70546
:1091600070E570B4060040047400F5702460022FAE
:1091700059B41226E57090C0FFF090BF2C122F82D8
:10918000A9701231EC90C0F5E013B390BF2DE054FC
:10919000F892E0122F82D24E80A3024AC2E55CB45C
:1091A00016030291A8B4141E124AB712788F90BF0A
:1091B0002DE05407B4060040027400F57012925B73
:1091C000755B040257D1B41506124AB702911DB45B
:1091D0000B29125CC4B45723124AB77E0312493DCF
:1091E0007400122F82125A4FDEF61250F2125609F4
:1091F00012493D12561B7466025CCF124AC2125CC1
:10920000C4B455111250F212560912493D12561BA0
:109210007457025CCFB456087457122F59025CC9B8
:1092200022E55CB4160302922CB41416124AB774E9
:1092300045122F597446125CCF12788F755B050268
:1092400057D1B4150302913DB41329124AB70570E2
:10925000E570B4060040047400F5702466122F59BE
:10926000E570B4050E124CFB7E0412868612788FD0
:1092700075700522B41222E570B4050E124AB77457
:109280006C122F59755B0802788F90BF2DE054F84F
:109290004570122F82D24E8093024AC2E55CB4160A
:1092A000030292A7B41416124AB712788F746E1282
:1092B0002F59746F125CCF755B060257D1B415033A
:1092C0000291A8B41128125CC4B48D061292D20285
:1092D00079E2124AB7E55EB40200400812497ED234
:1092E0005B0257D1D25F125D5E7446022F59B412F1
:1092F00026305F03122E837C07785E90BED1124B1E
:109300008A125CA7125D5E7447122F59125D5ED2FD
:109310005F755B09024AB7B40B005020305F08C28A
:109320005F122E831249F9E55E640B600F1260DC58
:10933000D267755D1A755A08755B0522024AC2E547
:109340005CB4160302934AB41416124AB712788F0B
:10935000745D122F59745E125CCF755B070257D192
:10936000B4150302922CB41126125CC4B48D0612FB
:1093700093750279E21570E5707002D25F124AB7F8
:10938000124A9E7400F6305F030250FC0280C5B49E
:10939000120F205FB5787190BF6CAC70124B8A8051
:1093A000A9A870B804005052F9B90A0579000293CF
:1093B000E09093B9E57025E07380088016801C80EA
:1093C000028008B9020040180293FAB90300401065
:1093D0000293FAB9040040080293FAB90500501A42
:1093E000305F0AC25F746F122F59125CC9124A9E15
:1093F000E9F60570122EAB024AB7124AC2125CD6C9
:10940000B46F1C122F5990BF6C7C04E0122DFC121B
:109410002EAD122E01125A4FDCF17470025CCFB4E3
:109420007006122F59025CC922E55CB4160302943F
:1094300034B41406124AB702911DB415030292A760
:10944000B41129125CC4B48D0612944F0279E21251
:109450004AB775F00078707971E6122E601570E5E4
:1094600070700612788F0250E80280C5B41208208E
:109470005FC212842980BD125CC4B45D0D124AC261
:10948000745E122F59745F025CCFB45E1F124AC221
:10949000745F122F59125CC9790190BF5FE0FEE939
:1094A000122E8A122EAD09DEF602788F124937404D
:1094B00003024AC2305F05C25F1250B6E57064080D
:1094C00060EF124AB7122EAB79717870E6855CF0C6
:1094D000122E600622E55CB4160302922CB414032B
:1094E00002922CB41503029242B4112B125CC4B444
:1094F0008D061294F80279E2124AB77F08787879DB
:1095000079124D7077001570E570700812788F74BD
:109510006C022F590280C5B4124E124AB7205F2840
:10952000128234E57679E87803124D64E575791096
:109530007827124D6412824290BF2EED547F122F75
:1095400082125A4FEE122F8275700590BF2DE05493
:10955000F84570122F82D24EE57012925B7445125C
:109560005CCF755B0502788FB40B00502B305F0821
:10957000C25F7570001250F7E570B4050050191203
:109580002EAB7F0878727971123023E55CB40A0241
:109590007400F70570024AB7024AC2E55CB41603CC
:1095A0000292A7B414030292A7B415030291A8B4BF
:1095B0001128125CC4B48D061295BE0279E2124ADB
:1095C000B7E55EB40200400812497ED25B0257D173
:1095D000D25F125D5E7447022F59B41216205FC627
:1095E0007C08785F90BEC7124B8A125C8A125D5E5F
:1095F0000292A7B40B00501D305F05C25F122F58B6
:10960000E55E6410600F1260DCD267755D1A755AF2
:1096100008755B0922024AC2E55CB4160302962370
:10962000B41403028C6AB41503028BEBB4110F124D
:109630005CC4B48D06128A4C0279E2028A46B412E6
:109640002AE570B40900404F90BEDF7871E6540FF0
:10965000122F8208125A4F7C04E6C408D6122F82B9
:10966000125A4F08DCF3124AB780B8B40B005027E7
:10967000E570B409005020B405028003B4030574FA
:109680002D122F4A122EAB7F087872797112302377
:10969000A75C0570024AB7024AC2E55B9096A20237
:1096A0000B6C0296AE0296D50296D50296D5125C48
:1096B000B8700EE55CB40D1CC23AC263D254024CC1
:1096C000091248ED79791278AB70091257BA1278FD
:1096D0008F02510B22E55CB40E0302637D22E55B31
:1096E0009096E6020B6C0296F20297790297E502D9
:1096F0009827306F7EC26F12986379DAF76074B47E
:109700000C59124ACE305F0C78CDB60D004005766C
:109710000002979378CD7600E55E603490BEB7E0A6
:1097200024CD125A94E55EC3133400B410005001E6
:1097300004FE785FE066700808125A4FDEF6800D6E
:1097400090BEB7E004122F8224CD1259D5125D5E6F
:10975000125CB87003024C14024C17B40B0CC25FBD
:10976000124ACE78CD7610025D5EC25F78CD76105B
:10977000022E2E78CDE660D522306F68C26F129827
:109780006379DAF7605EB40C2B124ACE78CDE660CE
:1097900013760012788F125CB8700574A9122F59D5
:1097A000755B0222E55E60071259C078CD7603D260
:1097B0005F024C14B40B09124ACE125D5E02510BCB
:1097C000125CC46007122F5878CD7600E55EB42095
:1097D000004005747F122F4A79DAE7122E2E79DACB
:1097E000E7022EAD22306F3EC26F12986379DAF72E
:1097F00060347F087872797112302379DAE7F5796D
:10980000057090BF5FE06570701C79791278AB705D
:1098100007124ACE755B032212788F125CB8700370
:10982000024C14024C1722306F38C26F12986379C1
:10983000DAF76023304618B40215124ACED254C269
:1098400063C23AC246E490BEB9122F82029857B45E
:109850000505C265028C3D125CB87003024C14020F
:109860004C172290D002E0540F90986E9322010280
:10987000030004050600070809000B0A0C00E55C5C
:10988000B400030298FFE55DB4180122E55CB43F23
:10989000030298FFB40B005003029BA8B4300040B1
:1098A00004540F241EC3940B9098AE020B6C029BC1
:1098B000A8029BA8029BA8029BA8029BA8029BA8A7
:1098C000029C1C029BA8029BA9029CE4029CE4024D
:1098D0009D98029BA8029BA8029BA8029BA8029BA2
:1098E000A9029D98029BA8029DC8029DC8029DC81E
:1098F000029DC8029DC8029DC8029DC8029DC878ED
:10990000CAE6701C20531990BF74E020E112306A3F
:109910000F1257EE6006306207207704C26AD24702
:109920001257EA701C105E03029A9CE55DB419039D
:10993000029944B41503029944125CB86006755D3F
:1099400018029A9C125CD6706CE55DB40A12124C37
:1099500017306006125183029A8D12511A029A8DA5
:10996000B41C0612511A029A8DB4063890C085E0D4
:10997000B40A027400126B0E4021C248305916908E
:10998000C05EE0655E7008055E126AB1029A7512EB
:109990006A9B029A8D126A89029A8D126AFD305E64
:1099A000F7029A75B40705124DAA80C9124E2C12FF
:1099B000511A029A8DB48206127D57029A75B483A9
:1099C00009122F59127D80029A75B4B00B122F59CB
:1099D0007431127C3B029A75B43110E55DB41906FE
:1099E000127F90029A8D7431029A8AB421061285F0
:1099F0006E029A8DB40406127D6D029A75B49906B2
:109A0000127D80029A75B4050B122F597457127B80
:109A1000D0029A75B4060B122F597421127EFD02E2
:109A20009A75B43B0ED267755D1A755A01755B0065
:109A3000029A8AB45615122F5912560912493D122C
:109A4000561B1292101257E5029A9CB45E061294AD
:109A500080029A75B45F06129490029A8DB44506FE
:109A600012922F029A75B466061291AB029A8DB4C7
:109A70006F091293FD1257DB029A9CB48C0612797F
:109A8000E5029A8DB4CA03124965122F59125CC9B6
:109A9000205C05124930700478C87615E55DB41372
:109AA000051275B88013B41C10E55BB40205126F83
:109AB000DA8006B4030312703B78C8B6001A205E41
:109AC00017205C1520533820520E20515E20630869
:109AD000E55DB400032054622278C87605125CC4A8
:109AE000648D600DE55DB41503755D00748D122FF6
:109AF00059124E4690C095E0122ED50214972212AC
:109B00004C17C251125CB8701A125CC4B4CA01225C
:109B100064C860FB74C8122F59742C122F4A740148
:109B2000122F52206DE9D26DD2472278C8760A12E0
:109B30005CC464186003025CEA22304C0EE539B460
:109B40008000400790C08DE010E40122F0125CC458
:109B50006035B403028011B4A400401FB4A607E529
:109B600055540FB40C0250E320121C12511A125C0F
:109B7000C460057436122F61029B95B43503029BB5
:109B80008FB436C7029B9530120B7435122F5912C1
:109B90004E5A029BA27436125CBF124E427E0312D2
:109BA00051A990C091025631221257CC206439E558
:109BB0005DB41A29E55AB40723E55BB40A1E125CAA
:109BC000C4B42A03029BDC1257EAB40400500D12FD
:109BD0004BF11257EA70057605028FFE22B41CFC89
:109BE000E55BB402F7026FDAE55DB41E0280EDE5D5
:109BF0005B70E91257EAB4060050E1124BF11257BC
:109C0000EA70D97607E55DB41206124AB70274B855
:109C1000B4140302756BB413C30275B81257EA602B
:109C200003029CE3305D19C25DD25F125D5E124992
:109C300073124E2C206406124C170249A702656667
:109C4000105B03029CE3E55DB41103026566B41E7C
:109C50000BE55BB4000302761B029CE3B41A38E503
:109C60005AB4087FE55BB404077F08787202301BA2
:109C7000B405030292E4B40609205F671250FC02A7
:109C8000788FB4070612788F0250E8B40803029563
:109C90000CB4094F0295D0B4170EE55BB401030272
:109CA00086B5B4023E028726B41938E55BB40103D9
:109CB00002856EB40203028577B4030302858AB479
:109CC000040302859BB405030285B7B4060302852D
:109CD000D3B407030285EEB40803028627B4090350
:109CE00002866222125CC4B4CA691257EA706376B3
:109CF00003E557540723F99041EE93F8E9240193C3
:109D0000F5828883E054B8FFE55C6415601CEF20A1
:109D1000E72370107857B60203029D1FB60416D2CF
:109D2000E7029D35C39408029D35EF10E707B4386C
:109D30000050022408FFE054474F122F82E55D6473
:109D40001A600F12493060077400306502743B02DC
:109D50005CCF221257CCE55DB40917125CC4641BBA
:109D600060F078C7B6060050E9124BF1E670E302E6
:109D70006C41B41A12785A795BB60503029D82B61B
:109D80000816B7011380CBB41CC8E55BB40203020C
:109D90006FDAB403BD02703BE55DB41A2BE55AB42B
:109DA0000806E55B640160201257CCE554645960F5
:109DB00017E539B46000501078C7B6050050091295
:109DC0004BF1E67003025FCE22B40A005005C2D503
:109DD000029DDEB4BE0092D5B4D700B3401D909D65
:109DE000FCB464004006C39464909EC4C333F5F091
:109DF00093F8E5F00493F5828883C322B010B0296C
:109E0000B044B05DB078B091B0ACB0C5B0DEB0F9E0
:109E1000B112B12DB146B15FB17AB193B1AEB1C754
:109E2000B1E0B1FBB214B22FB248B261B27CB295CC
:109E3000B2B0B2C9B2E2B2FDB316B331B34AB36342
:109E4000B37EB397B3B2B3CBB3E4B3FFB418B433B8
:109E5000B44CB465B480B499B4B4B4CDB4E6B5012F
:109E6000B51AB535B54EB567B582B59BB5B6B5CFA4
:109E7000B5E8B603B61CB637B650B669B684B69D1B
:109E8000B6B8B6D1B6ECB705B71EB739B752B76D8D
:109E9000B786B79FB7BAB7D3B7EEB807B820B83B05
:109EA000B854B86FB888B8A1B8BCB8D5B8F0B9097B
:109EB000B922B93DB956B971B98AB9A3B9BEB9D7F2
:109EC000B9F2BA0BA010A029A044A05DA078A0917F
:109ED000A0ACA0C5A0DEA0F9A112A12DA146A15F52
:109EE000A17AA193A1AEA1C7A1E0A1FBA214A22FC8
:109EF000A248A261A27CA295A2B0A2C9A2E2A2FD40
:109F0000A316A331A34AA363A37EA397A3B2A3CBB3
:109F1000A3E4A3FFA418A433A44CA465A480A4992B
:109F2000A4B4A4CDA4E6A501A51AA535A54EA567A0
:109F3000A582A59BA5B6A5CFA5E8A603A61CA63716
:109F4000A650A669A684A69DA6B8A6D1A6ECA7058C
:109F5000A71EA739A752A76DA786A79FA7BAA7D301
:109F6000A7EEA807A820A83BA854A86FA888A8A176
:109F7000A8BCA8D5A8F0A909A922A93DA956A971EC
:109F8000A98AA9A3A9BEA9D7A9F2AA0BFFFFFFFF1F
:109F9000FFFFFFFFFFFFFFFFFFFFFFFFFFFFFFFFD1
:109FA000FFFFFFFFFFFFFFFFFFFFFFFFFFFFFFFFC1
:109FB000FFFFFFFFFFFFFFFFFFFFFFFFFFFFFFFFB1
:109FC000FFFFFFFFFFFFFFFFFFFFFFFFFFFFFFFFA1
:10FFF000FFFFFFFFFFFFFFFFFFFFFFFFFFFFFF57B9
:00000001FF
